:100000000C94E0010C9408340C9435340C940802E0
:100010000C9408020C9408020C9408020C94080238
:100020000C9408020C9408020C9408020C94F30639
:100030000C9408020C9408020C9408020C94080218
:100040000C9414330C9408020C9469060C94A506C5
:100050000C9408020C9408020C9408020C940802F8
:100060000C9408020C940802084AD73B3BCE016E60
:1000700084BCBFFDC12F3D6C74319ABD56833DDAFF
:100080003D00C77F11BED9E4BB4C3E916BAAAABE0E
:10009000000000803F05A84CCDB2D44EB93836A937
:1000A000020C50B9918688083CA6AAAA2ABE000074
:1000B00000803F0664EC1B3C04BC163E3BE5B93CAB
:1000C000C93C37C29E5A3D660498083EEA69AAAA0E
:1000D0003E000000803F2020BF0020BF00BF007C0A
:1000E0002020202020202020202020202020202010
:1000F00020202000C8202020202020202020202078
:1001000020C900C8202020202020202020202020BE
:10011000C97C00D820202020202020202020202042
:10012000D97C00C820202020202020202020202032
:10013000C97C00C820202020202020202020202032
:10014000C97C00206172737369006D696E6F706F96
:100150007364206C6962726570696C6F7400202032
:10016000202020BABBBCBDBE7C2020202020CACBD2
:10017000CCCDCE7C00626F6F74696E672075703A6B
:10018000EDF2F2F2F2F2F2F2F30063616C69627284
:100190006174657C7C6D6561737572656420616DE9
:1001A000703A20200063616C6962726174657C7CC6
:1001B0006D6561737572656420616D703A20200011
:1001C00063616C6962726174657C7C6D6561737575
:1001D00072656420766F6C743A2000626174746595
:1001E0007279207761726E696E6720007478706929
:1001F000642076616C756573006261726F2074654E
:100200006D700074656D7064697370200061637453
:100210006976652000706173736976650075617633
:1002200074616C6B20007365747570207363726504
:10023000656E7C7C7C004368617220446F6E650A49
:1002400000526561647920666F7220466F6E740A91
:100250000055706461746520436861725365740071
:1002600000407A10F35A00A0724E18090010A5D46D
:10027000E80000E87648170000E40B54020000CACA
:100280009A3B000000E1F505000080969800000010
:1002900040420F000000A08601000000102700006F
:1002A0000000E803000000006400000000000A00F5
:1002B000000000000100000000002C76D888DC67F8
:1002C0004F0823DFC1DFAE59E1B1B796E5E3E45350
:1002D000C63AE651997696E8E6C28426EB898C9B6D
:1002E00062ED407C6FFCEFBC9C9F40F2BAA56FA50D
:1002F000F490055A2AF75C936B6CF9676DC11BFC8F
:10030000E0E40D47FEF520E6B500D0ED902E0300A9
:10031000943577050080841E080000204E0A0000F6
:1003200000C80C333333330F986E12831141EF8DB5
:100330002114893BE65516CFFEE6DB18D1844B38F5
:100340001BF77C1D901DA4BBE424203284725E2226
:100350008100C9F124ECA1E53D276E616E00696E54
:10036000660000000000240027002A0000000000B2
:10037000250028002B000000000023002600290093
:10038000040404040404040402020202020203033B
:100390000303030301020408102040800102040843
:1003A00010200102040810200000000700020100D4
:1003B00000030406000000000000000074043A0876
:1003C00011241FBECFEFD8E0DEBFCDBF13E0A0E009
:1003D000B1E0E2E0F3E702C005900D92A03FB10763
:1003E000D9F716E0A0EFB3E001C01D92A33AB10720
:1003F000E1F713E0C0ECD3E004C02297FE010E94B5
:100400007B39CC3BD107C9F70E9444350C947F3926
:100410000C940000FA01AA27283051F1203181F113
:10042000E8946F936E7F6E5F7F4F8F4F9F4FAF4FFC
:10043000B1E03ED0B4E03CD0670F781F891F9A1F0F
:10044000A11D680F791F8A1F911DA11D6A0F711DC3
:10045000811D911DA11D20D009F468943F912AE0CF
:10046000269F11243019305D3193DEF6CF010895B7
:10047000462F4770405D4193B3E00FD0C9F7F6CFE8
:10048000462F4F70405D4A3318F0495D31FD4052B0
:10049000419302D0A9F7EACFB4E0A6959795879546
:1004A00077956795BA95C9F7009761057105089525
:1004B0009B01AC010A2E06945795479537952795D1
:1004C000BA95C9F7620F731F841F951FA01D089569
:1004D000283008F027E03327DA01990F311D87FD16
:1004E000916000966105710539F432602E5F3D938D
:1004F00030E32A95E1F708959F3F30F08038710589
:10050000610509F03C5F3C5F3D93913008F08068E5
:10051000911DDF93CF931F930F93FF92EF92192FAB
:10052000987F9695E92F96959695E90FFF27E654C3
:10053000FD4F99273327EE24FF24A701E7010590FB
:100540000894079428F4360FE71EF81E491F511D22
:10055000660F771F881F991F0694A1F705900794CF
:1005600028F4E70EF81E491F561FC11D770F881F7C
:10057000991F661F0694A1F70590079428F4F80EBA
:10058000491F561FC71FD11D880F991F661F771F50
:100590000694A1F70590079420F4490F561FC71F32
:1005A000D81F990F661F771F881F0694A9F784919B
:1005B0001095177041F0D695C79557954795F794C4
:1005C000E7941A95C1F7E0E6F2E06894159015916A
:1005D00035916591959105907FE27395E118F10A47
:1005E000430B560BC90BD009C0F7E10CF11E431F9A
:1005F000561FC91FD01D7EF4703311F48A95E6CFC3
:10060000E894015030F0080F0AF40027021708F4AC
:10061000202F2395022F7A3328F079E37D932A95B2
:10062000E9F710C07D932A9589F60694979567950A
:10063000379517951794E118F10A430B560BC90B20
:10064000D00998F023957E9173957A3308F070E382
:100650007C932013B8F77E9170617D9330F0839581
:1006600071E37D9370E32A95E1F71124EF90FF90F9
:100670000F911F91CF91DF91992787FD9095089554
:10068000CF93DF93BC018230910510F462E070E0FB
:10069000A091A106B091A206ED0140E050E0E0E09B
:1006A000F0E021C0888199818617970769F48A81D3
:1006B0009B81309719F09383828304C09093A206A4
:1006C0008093A106FE0134C06817790738F44115FC
:1006D000510519F08417950708F4AC01FE018A81D1
:1006E0009B819C01E9012097E9F641155105A9F18B
:1006F000CA01861B970B049708F4BA01E0E0F0E00A
:100700002AC08D919C91119784179507F9F464176D
:10071000750781F412968D919C911397309719F07B
:100720009383828304C09093A2068093A106FD0167
:1007300032964CC0CA01861B970BFD01E80FF91FCA
:100740006193719302978D939C9340C0FD018281C8
:1007500093819C01D9011097A1F680919F069091F9
:10076000A006892B41F480918C0290918D02909388
:10077000A00680939F0640918E0250918F024115F2
:10078000510541F44DB75EB780918A0290918B027A
:10079000481B590B20919F063091A006CA01821B6D
:1007A000930B8617970780F0AB014E5F5F4F84175E
:1007B000950750F0420F531F5093A00640939F0699
:1007C000F9016193719302C0E0E0F0E0CF01DF91A5
:1007D000CF910895CF93DF93009709F450C0EC01B7
:1007E00022971B821A82A091A106B091A2061097AF
:1007F00009F140E050E0AC17BD0708F1BB83AA83C4
:10080000FE0121913191E20FF31FAE17BF0779F47A
:100810008D919C911197280F391F2E5F3F4F39837F
:10082000288312968D919C9113979B838A834115FF
:10083000510571F4D093A206C093A10620C0129670
:100840008D919C911397AD01009711F0DC01D3CFEE
:10085000FA01D383C28321913191E20FF31FCE17A6
:10086000DF0769F488819981280F391F2E5F3F4F78
:10087000FA01318320838A819B8193838283DF9174
:10088000CF910895FC010590615070400110D8F798
:10089000809590958E0F9F1F0895FC0161507040C8
:1008A00001900110D8F7809590958E0F9F1F0895A5
:1008B0006EBD0DB407FEFDCF8EB508958DE061E0ED
:1008C0000E9462348BE061E00E9462348CE060E060
:1008D0000E9462348AE061E00E9462341CBC80E5C0
:1008E0008CBD8DB58EB5089580EF93E00E945E04B7
:1008F0000895FC011382128288EE93E0A0E0B0E03C
:1009000084839583A683B78385EA92E0918380836D
:100910000895FC018089803419F421E030E002C0A0
:1009200020E030E0C9010895FC01818990E008953C
:10093000FC016487458766874787089580E090E0DB
:10094000089580E090E0089580E090E00895089593
:10095000EF92FF921F93CF93DF93162F7A0186E0D9
:1009600060E00E94A13480EF93E060E00E945804B0
:1009700080EF93E060E00E94580480EF93E069E02C
:100980000E94580480EF93E0612F0E945804C0E059
:10099000D0E0F701EC0FFD1F108180EF93E06AE0DB
:1009A0000E94580480EF93E06C2F0E94580480EF5F
:1009B00093E06BE00E94580480EF93E0612F0E9467
:1009C00058042196C633D10521F780EF93E068E003
:1009D0000E94580480EF93E060EA0E94580480EF80
:1009E00093E060EA0E94580485FDF9CF80EF93E020
:1009F00060E00E94580480EF93E06CE00E9458048D
:100A000086E061E00E94A134DF91CF911F91FF90B9
:100A1000EF9008951F93CF93DF93EC01162F86E09C
:100A200060E00E94A13480EF93E060E00E945804EF
:100A3000112319F0113059F404C080EF93E0688954
:100A400004C068896C6180EF93E00E94580486E0DE
:100A500061E00E94A134DF91CF911F910895EF9240
:100A6000FF920F931F938EE1489F70011124E60EB1
:100A7000F11C86E060E00E94A13400EF13E0C801A1
:100A800065E00E945804C8016F2D0E945804C801F7
:100A900066E00E945804C8016E2D0E9458041F9100
:100AA0000F91FF90EF900895EF92FF920F931F9395
:100AB0007C0100EF13E0C80167E00E945804C80100
:100AC0006FEF0E94580486E061E00E94A134F701B4
:100AD00087858F5F87871F910F91FF90EF90089513
:100AE000EF92FF920F931F93FC01E7848EE1E89E43
:100AF000700111248685E80EF11C86E060E00E94FA
:100B0000A13400EF13E0C80164E00E945804C8015A
:100B100063E00E945804C80165E00E945804C801BF
:100B20006F2D0E945804C80166E00E945804C80155
:100B30006E2D0E9458041F910F91FF90EF90089521
:100B40001F93CF93DF93EC01162F6C3731F40E9483
:100B50005405CE010E9470050AC080EF93E067E063
:100B60000E94580480EF93E0612F0E94580481E0B6
:100B700090E0DF91CF911F9108950F931F9386E02E
:100B800060E00E94A13400EF13E0C80164E00E941D
:100B90005804C80164E00E94580486E061E00E94A5
:100BA000A1341F910F9108951F93CF93DF93EC0110
:100BB000188A16E0198B8FE896E060E973E00E94CE
:100BC0007432813049F480E4888B88E0898B86E038
:100BD00060E00E94A13402C0188A198B86E060E0B0
:100BE0000E94A134DF91CF911F9108950F931F931D
:100BF000CF93DF93EC0186E061E00E94623482E0F3
:100C000060E00E94623482E061E00E94A134CE0183
:100C10000E94D40586E060E00E94A13480EF93E05A
:100C20006CEE0E94580480EF93E06FEF0E9458042E
:100C3000182F80EF93E060E00E945804688962609A
:100C400080EF93E00E94580462E370E080E090E05F
:100C50000E946A3380EF93E06CE60E9458041F7E86
:100C600080EF93E0612F0E9458048889803419F046
:100C70000DE010E002C000E110E01092F2031092CB
:100C8000F10317C06091F1037091F203605F80EF90
:100C900093E00E94580480EF93E069E00E945804BA
:100CA0008091F1039091F20301969093F203809367
:100CB000F1038091F1039091F2038017910714F3EF
:100CC000CE0161E00E940A05DF91CF911F910F9143
:100CD00008951F920F920FB60F9211242F933F93F6
:100CE0004F938F939F93EF93FF934091C600209172
:100CF0007E0630917F062F5F3F4F80918206909154
:100D00008306282339238091800690918106281735
:100D1000390779F080917E0690917F06E0918406F4
:100D2000F0918506E80FF91F408330937F062093EA
:100D30007E06FF91EF919F918F914F913F912F915F
:100D40000F900FBE0F901F9018951F920F920FB625
:100D50000F9211242F933F938F939F93EF93FF93C1
:100D600020918806309189068091860690918706A9
:100D700028173907E9F08091880690918906E0915B
:100D80008C06F0918D06E80FF91F80818093C600D4
:100D90008091880690918906019620918A0630916B
:100DA0008B0682239323909389068093880610C034
:100DB0002091860630918706809188069091890659
:100DC0002817390729F48091C1008F7D8093C100D5
:100DD000FF91EF919F918F913F912F910F900FBEB7
:100DE0000F901F9018951F920F920FB60F9211241B
:100DF0008F939F938091B3049091B404892B51F009
:100E00008091B5049091B60401969093B6048093B6
:100E1000B50409C08091B7049091B80401969093ED
:100E2000B8048093B7049F918F910F900FBE0F90DD
:100E30001F901895CF93DF93482FEB018091000608
:100E4000833009F45DC0843028F48130C1F08230F1
:100E500058F50AC0853009F4D2C0853008F4A8C01E
:100E6000863009F0F2C0E9C04C3309F0EEC081E0F1
:100E700080930006488384EB8093FF05E6C0842FAF
:100E800090E0E091FF05F0E0E827F927ED54FD4FF1
:100E900020812093FF05887F9070809741F582E044
:100EA00080930006498329C0242F30E0E091FF059C
:100EB000F0E0E227F327ED54FD4F80818093FF059A
:100EC0008091FE058F5F8093FE05823018F43B838E
:100ED0002A83BBC0922F88272A813B81820F931FD0
:100EE0009B838A830A978F3F910521F018F0109217
:100EF0000006ABC083E0809300061092FE05A5C0FB
:100F0000E42FF0E08091FF0590E0E827F927ED5409
:100F1000FD4F80818093FF056091FE056F5F6093B8
:100F2000FE05623089F0633020F4613009F08DC035
:100F300006C0633091F0643009F087C022C0842F6E
:100F400090E0A0E0B0E018C0242F30E040E050E096
:100F5000542F432F322F222707C0242F30E040E0A8
:100F600050E0A901332722278C819D81AE81BF816A
:100F7000820F931FA41FB51F8C839D83AE83BF83F5
:100F800064C0242F30E040E050E0522F4427332744
:100F900022278C819D81AE81BF81820F931FA41F68
:100FA000B51F8C839D83AE83BF8360930006A5CF5E
:100FB000242F30E0E091FF05F0E0E227F327ED5425
:100FC000FD4F80818093FF058091FE058F5F8093A8
:100FD000FE05813019F08230C1F503C039872887BA
:100FE00034C0922F882728853985280F391F3987E3
:100FF00028878A819B810A97F1F085E07CCFE42FD6
:10100000F0E08091FF0590E0E827F927ED54FD4FCF
:1010100080818093FF052091FE052F5F2093FE05C0
:1010200030E0FB01E20FF31F41878A819B810A9721
:101030002817390750F086E05ECFC75FDE4F488340
:10104000C950D14087E08093000680910006873028
:1010500069F410920006C75FDE4F9091FF0588810A
:10106000C950D140981711F48A8101C080E0DF9106
:10107000CF9108958F92AF92CF92EF92FF920F93FC
:101080001F9389E794E060E045EC50E024EC30E009
:1010900000EC10E0B1ECEB2EF12CCC24C394A8E9C9
:1010A000AA2EF0E28F2E0E94E42B86E994E00E94A3
:1010B00079041092A9041092AA041092AB04109221
:1010C000AC041092AD041092AE041092AF041092D2
:1010D000B0041092B2041092B1041092A8041F91AF
:1010E0000F91FF90EF90CF90AF908F900895AF92B7
:1010F000BF92CF92DF92EF92FF920F931F93E090F7
:101100007A06F0907B0600917C0610917D068FE5B3
:1011100090E0A0E0B0E0E80EF91E0A1F1B1F0E943D
:101120005C336E157F058007910708F44EC0A090D0
:10113000DE04B090DF04C090E004D090E104C6016A
:10114000B50120E030E040E85FE30E94E437181684
:1011500094F5E0902606F09027060091280610915D
:1011600029060E945C3320917A0630917B064091DB
:101170007C0650917D06621B730B840B950B0E94BD
:10118000BA369B01AC01C601B5010E94EF3720E0E1
:1011900030E04AE754E40E9421369B01AC01C801CB
:1011A000B7010E94543560932606709327068093FA
:1011B0002806909329060E945C3360937A06709308
:1011C0007B0680937C0690937D061F910F91FF9084
:1011D000EF90DF90CF90BF90AF900895AF92BF9205
:1011E000DF92EF92FF920F931F93CF93DF938C01C7
:1011F0008091010680FDE4C0F801F08089E794E069
:101200006F2D0E94C52CE801C75FDE4FEF2DF0E087
:10121000ED54FD4F80818883F801F18089E794E0E7
:101220006F2D0E94C52CEF2DF0E0888190E0E8271B
:10123000F927ED54FD4F80818883F801F28089E71A
:1012400094E06F2D0E94C52CEF2DF0E0888190E096
:10125000E827F927ED54FD4F80818883F801F3805A
:1012600089E794E06F2D0E94C52CEF2DF0E0888176
:1012700090E0E827F927ED54FD4F80818883F8013D
:10128000F48089E794E06F2D0E94C52CEF2DF0E0EB
:10129000888190E0E827F927ED54FD4F808188830D
:1012A000F8012481358146815781232F342F452F22
:1012B0005527F22E89E794E0622F0E94C52CEF2D6E
:1012C000F0E0888190E0E827F927ED54FD4F808118
:1012D0008883F80124813581468157819A0144270A
:1012E0005527F22E89E794E0622F0E94C52CEF2D3E
:1012F000F0E0888190E0E827F927ED54FD4F8081E8
:101300008883F8012481358146815781252F332731
:1013100044275527F22E89E794E0622F0E94C52CBE
:10132000EF2DF0E0888190E0E827F927ED54FD4F9C
:101330008081888389E794E060E00E94C52CE88181
:10134000F0E0ED54FD4F8081888389E794E060E010
:101350000E94C52CE881F0E0ED54FD4F8081888328
:10136000F801828193810B9718F18AE0A82EB12CA5
:10137000A00EB11E750112C0F701D1907F0189E75F
:1013800094E06D2D0E94C52CED2DF0E0888190E059
:10139000E827F927ED54FD4F808188832E2D2A19E7
:1013A00030E0F801828193810A972817390720F3EA
:1013B000075F1E4F89E794E0F80160810E94C52C09
:1013C000DF91CF911F910F91FF90EF90DF90BF9031
:1013D000AF900895DF93CF93CDB7DEB7CA50D14019
:1013E0000FB6F894DEBF0FBECDBF2CE329836A830E
:1013F0002AE030E03C832B83FC0184819581A68127
:10140000B7818D839E83AF83B887CE0101960E94FA
:10141000EE08C65FDE4F0FB6F894DEBF0FBECDBF3D
:10142000CF91DF9108958FE896E06AE773E00E941C
:101430007432882331F586E696E6A6E6B0E480931A
:10144000030690930406A0930506B093060680E079
:1014500090E0A0E8BFE38093070690930806A0936E
:101460000906B0930A0688EE93E090930C068093E9
:101470000B0681E880930D068DE880930E068DEFB4
:1014800025C082E598EBAEE0B0E48093030690932C
:101490000406A0930506B093060685E89BEEA1E539
:1014A000B0E48093070690930806A0930906B093D2
:1014B0000A0680EA94E190930C0680930B068BEF6A
:1014C00080930D0686E680930E068AEF80930F06C2
:1014D0000895FF920F931F930FE816E0C8016CE781
:1014E00073E00E94743280935C06C8016EE773E07B
:1014F0000E94743280935D06C80160E873E00E9428
:10150000743280933606C8016EE873E00E9474322C
:1015100080935406C8016AE873E00E947432809395
:101520005206C80164E873E00E94743280935E063C
:10153000C80166E873E00E94743280935F06C801B8
:101540006CE873E00E94743280934406C80162E93B
:1015500073E00E94743280936006C80164E973E00E
:101560000E94743280934306C80164EF73E00E94C6
:101570007432F82EC80165EF73E00E947432382F80
:1015800020E02F0D311D3093380620933706C80117
:1015900066EF73E00E947432F82EC80167EF73E0C3
:1015A0000E947432382F20E02F0D311D30933C06FD
:1015B00020933B06C80168EF73E00E947432F82E56
:1015C000C80169EF73E00E947432382F20E02F0DBC
:1015D000311D30933A0620933906C8016BEF73E052
:1015E0000E947432809335061F910F91FF900895E9
:1015F000BC018FE896E00E94743208956091C8049F
:101600007091C9048091CA049091CB0420E030E02D
:1016100040E152E40E94EF3720E030E044EB53E435
:101620000E9421360E9452380E9489369B01255023
:10163000304037FF03C09B01215E3F4FAAE1B6E077
:10164000F901ED54FC4F80818C932F5F3F4F243282
:10165000310514F020E030E0119686E0A532B8079D
:1016600079F71C9208952F923F924F925F926F925A
:101670007F928F929F92AF92BF92CF92DF92EF9222
:10168000FF920F931F93DF93CF9300D000D000D031
:10169000CDB7DEB7182F662E2091BE043091BF045F
:1016A0002A35310530F0C9018D549F4F8935910598
:1016B000E8F437FF02C02D543F4FC90137FF03C084
:1016C000909581959F4F8A3191053CF0F4E48F2EDF
:1016D000912CE9ED2E2E312C1DC00A975CF17BE395
:1016E000872E912C62ED262E312C20C02B35310512
:1016F00014F0235B3040C90137FF03C090958195FA
:101700009F4F8A31910554F056E5852E912C4CED72
:10171000242E312C37E0A32EB12C15C00A9754F09B
:101720002DE4822E912C94ED292E312C88E0A82EC8
:10173000B12C09C005E0802E912CB8E32B2E312C62
:10174000A9E0AA2EB12C6091C0047091C104882731
:1017500077FD8095982F0E94BC3627EA32E94BE24C
:101760005CEB0E94EF370E94C33820E030E040EA93
:1017700050E40E94EF3720E030E040E951E40E945D
:10178000EF370E94523820E030E044E352E40E94F8
:1017900054350E948936712EFEEBCF2EFFEFDF2EDF
:1017A0009B01442737FD4095542F29833A834B836F
:1017B0005C83E6E94E2EE4E05E2E4AEF5FEF240EF6
:1017C000351E6091BE047091BF04882777FD809517
:1017D000982F0E94BC3625E33AEF4EE85CE30E9466
:1017E000EF370E94C3387B018C01B601882777FD53
:1017F0008095982F0E94BC369B01AC01C801B701AF
:101800000E94EF377B018C0169817A818B819C81F9
:101810000E94BC369B01AC01C801B7010E9454353F
:101820000E9489369B01CB0101978A35910508F00A
:1018300071C062E170E00E9415398B012F5F3F4F4C
:10184000AEEEBFEF6A9FC0016B9F900D7A9F900D27
:101850001124820F931F62E070E00E9415396D839E
:101860007E83E62CE01A4E2D4C5F86E994E0672DCE
:101870000E942F0500D000D000D0EDB7FEB7319602
:10188000ADB7BEB712965C924E92119720E031E050
:10189000338322838D819E81880D991D9583848356
:1018A0000E94C32B4DB75EB74A5F5F4F0FB6F894E7
:1018B0005EBF0FBE4DBF8D819E818A159B0554F181
:1018C000043011053CF593E0E90EC201672D4E2D61
:1018D0000E942F0500D000D000D0EDB7FEB73196A2
:1018E000ADB7BEB712965C924E92119720E031E0F0
:1018F000338322834D815E81420D531D5583448382
:101900000E94C32B8DB79EB706960FB6F8949EBF64
:101910000FBE8DBFACE0B0E0CA0EDB1E7394BEE418
:10192000CB16D10409F04DCF26960FB6F894DEBF42
:101930000FBECDBFCF91DF911F910F91FF90EF9020
:10194000DF90CF90BF90AF909F908F907F906F90DF
:101950005F904F903F902F900895823010F422E0D6
:1019600002C0282F220F30E08DB79EB708970FB620
:10197000F8949EBF0FBE8DBFEDB7FEB7319686E9D6
:1019800094E0ADB7BEB712969C938E93119783E007
:1019900091E09383828322573F4F358324832F5FC7
:1019A0003F4F378326830E94C32B8DB79EB708967F
:1019B0000FB6F8949EBF0FBE8DBF0895CF93DF93EF
:1019C000AC01E091D004F091D10420911006309147
:1019D0001106C9018C599F4F8E179F071CF4EA010D
:1019E000219709C024563040E217F30714F0EA01AA
:1019F00002C0EA012196842F90E0C817D90729F088
:101A00008FE896E04C2F0E947B32CE01DF91CF9180
:101A100008950F931F930FE816E0C80163EF73E07A
:101A200041E00E947B32C80164EF73E043E10E9411
:101A30007B32C80165EF73E046E00E947B32C8014B
:101A400066EF73E040E10E947B32C80167EF73E00C
:101A500047E20E947B32C80168EF73E048E80E94C9
:101A60007B32C80169EF73E043E10E947B321F9132
:101A70000F910895CF92DF92EF92FF920F931F93F1
:101A8000CF93DF937C016B01EA0100D000D006E91F
:101A900014E0EDB7FEB7128301838FED90E09483DD
:101AA00083830E94B22B0F900F900F900F90CA303B
:101AB000D10581F0C436D10521F0C130D10519F529
:101AC00012C000D000D0EDB7FEB7128301838DEDB8
:101AD00090E011C000D000D0EDB7FEB712830183B3
:101AE0008AED90E008C000D000D0EDB7FEB71283B9
:101AF000018386ED90E0948383830E94B22B0F9044
:101B00000F900F900F904091D0045091D1042091EC
:101B1000100630911106C9018C599F4F8417950703
:101B20002CF4C7018C1B9D0BEC0109C024563040DE
:101B30004217530714F0E70114C0CE0DDF1DCE1578
:101B4000DF0579F08FE896E0B6014C2F0E947B32DA
:101B50000894C11CD11C8FE896E0B6014D2F0E945D
:101B60007B32CE01DF91CF911F910F91FF90EF90CB
:101B7000DF90CF900895CF92DF92EF92FF920F9374
:101B80001F937C01D62EC72E06E914E0C8016E2DE6
:101B90004D2D0E949804C8010E94700500D000D00D
:101BA000EDB7FEB71283018383E391E094838383CF
:101BB0000E94B22BEDB7FEB71283018383E291E05E
:101BC000948383830E94B22BEDB7FEB71283018307
:101BD00083E191E0948383830E94B22BEDB7FEB73B
:101BE0001283018383E091E0948383830E94B22B6C
:101BF000EDB7FEB71283018384EF90E09483838373
:101C00000E94B22B0F900F900F900F90C8010E946E
:101C10005405C70101966D2D7C2D0E94330B1F9139
:101C20000F91FF90EF90DF90CF900895AF92BF9209
:101C3000CF92DF92EF92FF920F931F93B82EA62EB2
:101C40000E945C3328EE33E040E050E00E942839E7
:101C500069017A0106E914E0C8016B2D4A2D0E9442
:101C60009804C8010E9470058DB79EB70C970FB6F7
:101C7000F8949EBF0FBE8DBFEDB7FEB73196ADB7DE
:101C8000BEB712961C930E93119788E091E0938350
:101C9000828383EB90E095838483C6016CE370E0DC
:101CA0000E941539CB016CE370E00E9415399783CF
:101CB00086838AE390E091878087C6016CE370E0B9
:101CC0000E941539938782870E94C32B8DB79EB7D8
:101CD0000C960FB6F8949EBF0FBE8DBFC8010E9430
:101CE00054051F910F91FF90EF90DF90CF90BF9020
:101CF000AF9008950F931F93282F462F06E914E005
:101D0000C801622F0E949804C8010E94700500D08B
:101D100000D0EDB7FEB71283018384E191E0948394
:101D200083830E94C32B0F900F900F900F90C801D8
:101D30000E9454051F910F9108958F929F92AF9228
:101D4000BF92CF92DF92EF92FF920F931F93E82EF4
:101D5000F62E06E914E0C8016E2D4F2D0E9498045E
:101D6000C8010E9470058DB79EB70C970FB6F89406
:101D70009EBF0FBE8DBFEDB7FEB73196ADB7BEB7F4
:101D800012961C930E9311978CE1882E81E0982E69
:101D900093828282BDEEAB2EB12CB582A48280915B
:101DA000E7049091E804A091E904B091EA048683E5
:101DB0009783A087B187A3EFCA2ED12CD386C28682
:101DC0000E94C32B8DB79EB70C960FB6F8949EBF9A
:101DD0000FBE8DBFC8010E945405F394C8016E2D3B
:101DE0004F2D0E949804C8010E947005ADB7BEB780
:101DF0001C970FB6F894BEBF0FBEADBFEDB7FEB7D0
:101E0000319612961C930E93119793828282B5821B
:101E1000A4828091EB049091EC04A091ED04B09128
:101E2000EE0486839783A087B187D386C2860E94FB
:101E3000C32B8DB79EB70C960FB6F8949EBF0FBEFE
:101E40008DBFC8010E945405F394C8016E2D4F2D1B
:101E50000E949804C8010E947005ADB7BEB71C97D8
:101E60000FB6F894BEBF0FBEADBFEDB7FEB731964B
:101E700012961C930E93119793828282B582A4824C
:101E80008091EF049091F004A091F104B091F204DC
:101E900086839783A087B187D386C2860E94C32B8F
:101EA0008DB79EB70C960FB6F8949EBF0FBE8DBF30
:101EB000C8010E9454051F910F91FF90EF90DF9091
:101EC000CF90BF90AF909F908F9008950F931F93E6
:101ED000282F462F06E914E0C801622F0E949804BB
:101EE000C8010E9470058DB79EB70A970FB6F89487
:101EF0009EBF0FBE8DBFEDB7FEB73196ADB7BEB773
:101F000012961C930E93119786E291E0938382833D
:101F100089EB90E09583848380911206909113065B
:101F20009783868382E890E0918780870E94C32B05
:101F30008DB79EB70A960FB6F8949EBF0FBE8DBFA1
:101F4000C8010E9454051F910F910895EF92FF92CE
:101F50000F931F93282F462F96E9E92E94E0F92E30
:101F6000C701622F0E949804C7010E9470058DB7B7
:101F70009EB70C970FB6F8949EBF0FBE8DBF0DB7DE
:101F80001EB70F5F1F4FEDB7FEB7F282E1828EE200
:101F900091E0F8019383828384EE90E095838483BB
:101FA0006091140670911506882777FD8095982F0B
:101FB0000E94BC362AE037ED43E25CE30E94EF3733
:101FC000F80166837783808791878FE890E0938715
:101FD00082870E94C32B8DB79EB70C960FB6F894DC
:101FE0009EBF0FBE8DBFC7010E9454051F910F9168
:101FF000FF90EF9008950F931F93282F462F06E927
:1020000014E0C801622F0E949804C8010E94700564
:102010008DB79EB70C970FB6F8949EBF0FBE8DBFBD
:10202000EDB7FEB73196ADB7BEB712961C930E93BF
:1020300011978EE291E09383828382EE90E0958304
:1020400084838091160690911706A0911806B0918E
:10205000190686839783A087B1878EE890E09387DF
:1020600082870E94C32B8DB79EB70C960FB6F8944B
:102070009EBF0FBE8DBFC8010E9454051F910F91D6
:1020800008950F931F93282F462F86E994E0622F1F
:102090000E94980486E994E00E9470058091CD0426
:1020A000882319F428E331E057C0813019F42CE378
:1020B00031E052C0823019F420E431E04DC0833069
:1020C00019F424E431E048C0843019F428E431E004
:1020D00043C0853019F42CE431E03EC0863019F459
:1020E00020E531E039C0873019F424E531E034C00F
:1020F000883019F428E531E02FC0893019F42CE537
:1021000031E02AC08A3019F420E631E025C08B3056
:1021100019F424E631E020C08C3019F428E631E0CF
:102120001BC08D3019F42CE631E016C08E3019F446
:1021300020E731E011C08F3019F424E731E00CC002
:10214000803119F428E731E007C0813119F02CE71C
:1021500031E002C02DE731E08DB79EB708970FB68A
:10216000F8949EBF0FBE8DBFEDB7FEB7319606E95E
:1021700014E0ADB7BEB712961C930E93119781E889
:1021800091E09383828380EE90E09583848337830C
:1021900026830E94C32B8DB79EB708960FB6F8947E
:1021A0009EBF0FBE8DBFC8010E9454051F910F91A5
:1021B00008950F931F93282F462F06E914E0C801B6
:1021C000622F0E949804C8010E9470058DB79EB7C7
:1021D0000A970FB6F8949EBF0FBE8DBFEDB7FEB73E
:1021E0003196ADB7BEB712961C930E93119786E841
:1021F00091E09383828387E890E095838483809144
:10220000CE049091CF049783868385E290E09187F6
:1022100080870E94C32B8DB79EB70A960FB6F8949D
:102220009EBF0FBE8DBFC8010E9454051F910F9124
:1022300008950F931F93282F462F06E914E0C80135
:10224000622F0E949804C8010E9470058DB79EB746
:102250000A970FB6F8949EBF0FBE8DBFEDB7FEB7BD
:102260003196ADB7BEB712961C930E93119780E9C5
:1022700091E0938382838091C0049091C1049583FF
:10228000848380EB90E09783868381EB90E0918755
:1022900080870E94C32B8DB79EB70A960FB6F8941D
:1022A0009EBF0FBE8DBFC8010E9454051F910F91A4
:1022B00008950F931F93282F462F06E914E0C801B5
:1022C000622F0E949804C8010E9470058DB79EB7C6
:1022D0000A970FB6F8949EBF0FBE8DBFEDB7FEB73D
:1022E0003196ADB7BEB712961C930E93119780E945
:1022F00091E0938382838091BE049091BF04958383
:10230000848380EB90E09783868382EB90E09187D3
:1023100080870E94C32B8DB79EB70A960FB6F8949C
:102320009EBF0FBE8DBFC8010E9454051F910F9123
:1023300008950F931F93282F462F06E914E0C80134
:10234000622F0E949804C8010E9470058DB79EB745
:102350000A970FB6F8949EBF0FBE8DBFEDB7FEB7BC
:102360003196ADB7BEB712961C930E93119788E9BC
:1023700091E09383828381EE90E0958384838091C2
:102380009802909199029783868385E290E09187E5
:1023900080870E94C32B8DB79EB70A960FB6F8941C
:1023A0009EBF0FBE8DBFC8010E9454051F910F91A3
:1023B00008950F931F93282F462F06E914E0C801B4
:1023C000622F0E949804C8010E9470058DB79EB7C5
:1023D0000C970FB6F8949EBF0FBE8DBFEDB7FEB73A
:1023E0003196ADB7BEB712961C930E93119780EA43
:1023F00091E0938382838AEA91E09583848380EDE0
:1024000090E0978386838AE196E09187808781EDCB
:1024100090E0938782870E94C32B8DB79EB70C965E
:102420000FB6F8949EBF0FBE8DBFC8010E94540521
:102430001F910F9108950F931F93282F462F06E9A0
:1024400014E0C801622F0E949804C8010E94700520
:102450008DB79EB70A970FB6F8949EBF0FBE8DBF7B
:10246000EDB7FEB73196ADB7BEB712961C930E937B
:10247000119788EB91E0938382838091C8049091B7
:10248000C904A091CA04B091CB0484839583A68328
:10249000B78380EB90E0918780870E94C32B8DB734
:1024A0009EB70A960FB6F8949EBF0FBE8DBFC801A7
:1024B0000E9454051F910F9108950F931F93282F89
:1024C000462F06E914E0C801622F0E949804C80153
:1024D0000E9470058DB79EB70C970FB6F8949EBFFB
:1024E0000FBE8DBFEDB7FEB73196ADB7BEB7129632
:1024F0001C930E93119780EC91E09383828386E185
:1025000090E0958384838091E2049091E304A0910C
:10251000E404B091E50486839783A087B18788E8B7
:1025200090E0938782870E94C32B8DB79EB70C964D
:102530000FB6F8949EBF0FBE8DBFC8010E94540510
:102540001F910F910895EF92FF920F931F93282FE1
:10255000462F36E9E32E34E0F32EC701622F0E94A6
:102560009804C7010E9470058DB79EB70C970FB6EF
:10257000F8949EBF0FBE8DBF0DB71EB70F5F1F4FE4
:10258000EDB7FEB7F282E18280EC91E0F80193832F
:10259000828389EE90E0958384836091DE0470915C
:1025A000DF048091E0049091E104209103063091D2
:1025B000040640910506509106060E94EF37F80187
:1025C000668377838087918780910D068287138643
:1025D0000E94C32B8DB79EB70C960FB6F8949EBF82
:1025E0000FBE8DBFC7010E9454051F910F91FF9030
:1025F000EF900895EF92FF920F931F93282F462F8D
:1026000056E9E52E54E0F52EC701622F0E9498048A
:10261000C7010E9470058DB79EB70C970FB6F8944E
:102620009EBF0FBE8DBF0DB71EB70F5F1F4FEDB71B
:10263000FEB7F282E1828AEC91E0F8019383828313
:1026400086EE90E0958384836091DA047091DB04D8
:102650008091DC049091DD042091070630910806FA
:102660004091090650910A060E94EF37F8016683EF
:1026700077838087918780910E06828713860E94D8
:10268000C32B8DB79EB70C960FB6F8949EBF0FBEA6
:102690008DBFC7010E9454051F910F91FF90EF90CD
:1026A0000895EF92FF920F931F93282F462F66E90C
:1026B000E62E64E0F62EC701622F0E949804C7013F
:1026C0000E9470058DB79EB70C970FB6F8949EBF09
:1026D0000FBE8DBF0DB71EB70F5F1F4FEDB7FEB713
:1026E000F282E1828AEC91E0F8019383828387EEA3
:1026F00090E0958384836091DA047091DB0480918B
:10270000DC049091DD0420912A0630912B06409143
:102710002C0650912D060E945335209107063091CA
:1027200008064091090650910A060E94EF37F80109
:10273000668377838087918780910E0682871386D0
:102740000E94C32B8DB79EB70C960FB6F8949EBF10
:102750000FBE8DBFC7010E9454051F910F91FF90BE
:10276000EF9008950F931F93282F462F06E914E04A
:10277000C801622F0E949804C8010E9470058091D0
:102780002E060E94AD0CC8010E9454051F910F91A6
:102790000895EF92FF920F931F93282F462F76E90B
:1027A000E72E74E0F72EC701622F0E949804C7013C
:1027B0000E9470058DB79EB70C970FB6F8949EBF18
:1027C0000FBE8DBF0DB71EB70F5F1F4FEDB7FEB722
:1027D000F282E1828AEC91E0F801938382838FE1B7
:1027E00090E09583848360912F06709130068091EC
:1027F0003106909132060E94BC3620910706309136
:1028000008064091090650910A060E94EF37F80128
:10281000668377838087918780910E0682871386EF
:102820000E94C32B8DB79EB70C960FB6F8949EBF2F
:102830000FBE8DBFC7010E9454051F910F91FF90DD
:10284000EF9008950F931F93282F462F06E914E069
:10285000C801622F0E949804C8010E9470058DB7BC
:102860009EB740970FB6F8949EBF0FBE8DBFEDB7D1
:10287000FEB73196ADB7BEB712961C930E93119763
:1028800084ED91E09383828383E890E09583848351
:102890008091C4049091C504A091C604B091C7046E
:1028A00086839783A087B18784E890E093878287A7
:1028B0008091D4049091D504A091D604B091D7040E
:1028C00084879587A687B7870E94C32B8DB79EB74D
:1028D00040960FB6F8949EBF0FBE8DBFC8010E94F0
:1028E00054051F910F9108950F931F93282F462F82
:1028F00086E994E0622F0E94980486E994E00E94A1
:1029000070058091D904282F30E0823030F4E4E063
:10291000220F331FEA95E1F702C02150304000D06A
:1029200000D000D0EDB7FEB7319606E914E0ADB7A0
:10293000BEB712961C930E93119780E091E093839B
:102940008283358324830E94C32B8DB79EB706965E
:102950000FB6F8949EBF0FBE8DBFC8010E945405EC
:102960001F910F9108950F931F93282F462F06E96B
:1029700014E0C801622F0E949804C8010E947005EB
:102980008DB79EB708970FB6F8949EBF0FBE8DBF48
:10299000EDB7FEB73196ADB7BEB712961C930E9346
:1029A000119786EE91E0938382838FE090E0958388
:1029B00084838091D804868317820E94C32B8DB7AD
:1029C0009EB708960FB6F8949EBF0FBE8DBFC80184
:1029D0000E9454051F910F9108950F931F9306E9CC
:1029E00014E0C80163E045E00E949804C8010E9419
:1029F000700500D000D0EDB7FEB7128301838EE5DD
:102A000091E0948383830E94B22BEDB7FEB71283CB
:102A100001838AE491E0948383830E94B22BEDB713
:102A2000FEB71283018383E491E0948383830E9441
:102A3000B22B0F900F900F900F90C8010E94540579
:102A40001F910F9108950F931F93282F462F06E98A
:102A500014E0C801622F0E949804C8010E9470050A
:102A600000D000D0EDB7FEB71283018385E791E077
:102A7000948383830E94B22B0F900F900F900F903E
:102A8000C8010E9454051F910F910895EF92FF9283
:102A90000F931F93CF93DF930E945C3320913E06E8
:102AA00030913F0640914006509141062617370766
:102AB0004807590708F04FC30E945C336C507E4FA3
:102AC0008F4F9F4F60933E0670933F068093400662
:102AD0009093410606E914E0C8010E94BD05C801B3
:102AE00065E043E00E949804C8010E94700500D090
:102AF00000D0ADB7BEB712961C930E93119786E225
:102B000092E014969C938E9313970E94B22B0F9091
:102B10000F900F900F908091100690911106892BC5
:102B200031F08091330690913406892B81F48091A5
:102B3000D0049091D1049093110680931006809157
:102B4000D2049091D304909334068093330620915D
:102B5000D2043091D3044091330650913406C90118
:102B6000845690404817590724F480913D068F5FA2
:102B700008C02C593F4F241735072CF480913D068F
:102B8000815080933D0680913D06181614F081E037
:102B900003C08D301CF08CE080933D0680913D0693
:102BA000863009F45AC187308CF4833009F4FAC0B6
:102BB000843034F4813079F1823009F0C8C28BC09E
:102BC0008430E9F0853009F0C2C222C0893009F4AE
:102BD000B7C18A3034F4873079F0883009F0B7C251
:102BE00014C08B3079F08B3024F08C3009F0AFC2F8
:102BF0002BC2C4E6D0E02FC2C4E6D0E0A8C1C4E630
:102C0000D0E032C184E690E021C284E690E09AC12F
:102C100084E690E024C100D000D0C6E9D4E0EDB74E
:102C2000FEB7D283C1838DE192E0948383830E94B7
:102C3000B22B809101060F900F900F900F9080FFA4
:102C400026C000D000D0ADB7BEB71296DC93CE93AD
:102C5000119785E192E014969C938E9313970E94AE
:102C6000B22B8091100690911106845690400F90DF
:102C70000F900F900F902091D0043091D10428171D
:102C800039070CF064C2809101068E7F21C000D00C
:102C900000D0EDB7FEB7D283C1838DE092E094837C
:102CA00083830E94B22B80911006909111068C595B
:102CB0009F4F0F900F900F900F902091D004309164
:102CC000D104821793070CF042C280910106816003
:102CD000809301063CC200D000D0C6E9D4E0ADB775
:102CE000BEB71296DC93CE93119783E092E01496D0
:102CF0009C938E9313970E94B22B0F900F900F907E
:102D00000F9080913506882301F100D000D0EDB7F7
:102D1000FEB7D283C18389EF91E0948383830E94BD
:102D2000B22B8091100690911106845690400F901E
:102D30000F900F900F902091D0043091D10428175C
:102D400039073CF51092350624C000D000D0ADB74D
:102D5000BEB71296DC93CE9311978CEE91E0149649
:102D60009C938E9313970E94B22B809110069091A2
:102D700011068C599F4F0F900F900F900F9020913C
:102D8000D0043091D104821793071CF481E0809322
:102D900035068FE896E06BEF73E0409135060E94B0
:102DA0007B32D5C100D000D0B6E9EB2EB4E0FB2ECB
:102DB000EDB7FEB7F282E1828BED91E094838383DD
:102DC0000E94B22B8DB79EB708970FB6F8949EBF9E
:102DD0000FBE8DBF0DB71EB70F5F1F4FADB7BEB78C
:102DE0001296FC92EE9211978CEE91E0F80193838B
:102DF00082836091360670E080E090E00E94BA36EF
:102E000020E030E040E251E40E942136D8011496DF
:102E10006D937D938D939C93179786E790E0199619
:102E20009C938E93189780E290E01B969C938E93D0
:102E30001A970E94C32BEDB7FEB73C960FB6F894D5
:102E4000FEBF0FBEEDBF8091360690E060E873E0F4
:102E50000E94DE0C809336067AC18AE090E06AE038
:102E600070E00E941539EB0100D000D006E914E0B3
:102E7000ADB7BEB712961C930E93119780EC91E0FC
:102E800014969C938E9313970E94B22BEDB7FEB7C6
:102E900038970FB6F894FEBF0FBEEDBF3196ADB7B1
:102EA000BEB712961C930E9311978EE291E0938316
:102EB000828382EE90E095838483809116069091C0
:102EC0001706A0911806B091190686839783A087EC
:102ED000B1878EE890E0938782870E94C32BEDB77D
:102EE000FEB736960FB6F894FEBF0FBEEDBF319613
:102EF000ADB7BEB712961C930E93119784EF91E075
:102F000093838283809137069091380695838483DA
:102F10000E94C32BEDB7FEB736960FB6F894FEBFEE
:102F20000FBEEDBF809137069091380664EF73E0D5
:102F3000AE010E943A0D909338068093370607C180
:102F40008AE090E06AE070E00E941539EB0100D061
:102F500000D0A6E9EA2EA4E0FA2EADB7BEB71296CD
:102F6000FC92EE92119785EA91E014969C938E93D1
:102F700013970E94B22BEDB7FEB738970FB6F894AF
:102F8000FEBF0FBEEDBF0DB71EB70F5F1F4FF28222
:102F9000E1828EE291E0D80113969C938E93129772
:102FA00084EE90E015969C938E931497609114068E
:102FB00070911506882777FD8095982F0E94BC3662
:102FC0002AE037ED43E25CE30E94EF37F8016683C5
:102FD0007783808791878FE890E0938782870E942C
:102FE000C32B8DB79EB706960FB6F8949EBF0FBE43
:102FF0008DBFEDB7FEB73196ADB7BEB71296FC9256
:10300000EE9211978BE092E0938382838091390650
:1030100090913A06958384830E94C32BEDB7FEB747
:1030200036960FB6F894FEBF0FBEEDBF80913906FD
:1030300090913A0668EF73E0AE010E943A0D9093CA
:103040003A068093390683C08AE090E06AE070E037
:103050000E941539EB0100D000D0F6E9EF2EF4E024
:10306000FF2EADB7BEB71296FC92EE9211978AE88A
:1030700091E014969C938E9313970E94B22BEDB718
:10308000FEB738970FB6F894FEBF0FBEEDBF0DB771
:103090001EB70F5F1F4FF282E1828EE291E0D801EE
:1030A00013969C938E93129784EE90E015969C93C2
:1030B0008E9314976091140670911506882777FDFA
:1030C0008095982F0E94BC362AE037ED43E25CE3FE
:1030D0000E94EF37F80166837783808791878FE8B6
:1030E00090E0938782870E94C32B8DB79EB7069688
:1030F0000FB6F8949EBF0FBE8DBFEDB7FEB73196E9
:10310000ADB7BEB71296FC92EE92119782E292E0B2
:103110009383828380913B0690913C0695838483C0
:103120000E94C32BEDB7FEB736960FB6F894FEBFDC
:103130000FBEEDBF80913B0690913C0666EF73E0B9
:10314000AE010E943A0D90933C0680933B0686E9BF
:1031500094E00E945405DF91CF911F910F91FF9051
:10316000EF9008952F923F924F925F926F927F92CD
:103170008F929F92AF92BF92CF92DF92EF92FF9287
:103180000F931F93DF93CF93CDB7DEB729970FB679
:10319000F894DEBF0FBECDBF8E836F830E945C3379
:1031A00020914B0630914C0640914D0650914E06B1
:1031B000261737074807590708F02BC180914F069B
:1031C0008823C9F080939A0210924F0689E392E017
:1031D00090935106809350060E945C336C507E4F52
:1031E0008F4F9F4F60934B0670934C0680934D0614
:1031F00090934E06C9C080919A02482E5524809122
:10320000CC048D8300915006109151069091B90421
:103210009983A091D904AC83B0914206BB8380907E
:10322000160690901706A0901806B0901906909177
:103230003606609098027090990280914306282E7D
:103240003324E0914406EA8359864886C92EDD245A
:10325000EE24FF24888599850196998788870697AB
:103260002CF0A1E0B0E0B987A88718C0E885F985FF
:10327000E330F10509F1E430F1053CF4E130F1050A
:1032800069F0329709F047C010C08885998584306D
:103290009105E1F0059709F03EC02EC09D81923066
:1032A000D0F506E412E081E03DC0A981A33099F198
:1032B00003E512E082E036C0BC81B23060F5EB81FC
:1032C000EE2349F100E612E083E02CC0C701B6010D
:1032D0000E94BA3620E030E040E251E40E942136FC
:1032E0009B01AC01C501B4010E941A3688239CF4ED
:1032F0000DE612E084E016C06214730464F4FDE984
:103300006F16FFEF7F0639F08A81882321F40AE7E0
:1033100012E085E007C0A885B985A415B50509F0B8
:1033200099CF60C0109351060093500680934F06CA
:1033300081E0809345060E945C3368517C4F8F4F3B
:103340009F4F60934B0670934C0680934D0690936D
:103350004E060E945C336056704F8F4F9F4F6093B4
:103360004706709348068093490690934A068091D9
:103370004606882321F086E994E00E94BD0510925C
:10338000460602C01092450606E914E0C8016E81A7
:103390004F810E949804C8010E94700500D000D09F
:1033A00000D0EDB7FEB73196ADB7BEB712961C93FD
:1033B0000E93119787E892E0938382838091500661
:1033C00090915106958384830E94C32BEDB7FEB77D
:1033D00036960FB6F894FEBF0FBEEDBFC8010E942F
:1033E000540517C0109351060093500610924F06D3
:1033F0000E945C332091470630914806409149066F
:1034000050914A06261737074807590708F4BACFDC
:10341000BBCF29960FB6F894DEBF0FBECDBFCF91BC
:10342000DF911F910F91FF90EF90DF90CF90BF90B1
:10343000AF909F908F907F906F905F904F903F9054
:103440002F900895EF92FF920F931F938091520651
:10345000843009F056C09091CD04943008F027C113
:1034600080915B068917A1F190935B060E945C3303
:1034700060935706709358068093590690935A06A6
:1034800090915B0680919B02981711F580914606FA
:10349000813091F0813018F08230B1F413C011E026
:1034A000109346060E945C336153754780409040FC
:1034B00030F41093530608C082E0809346061092C1
:1034C000530602C01092460686E994E00E94BD05AC
:1034D0000E945C332091570630915806409159065E
:1034E00050915A06621B730B840B950B615D7740FC
:1034F0008040904008F4DBC08091CD0480939B0213
:10350000D6C0853029F4809190029091910214C028
:10351000863029F480919202909193020DC08730F9
:1035200029F4809194029091950206C0883041F46C
:10353000809196029091970290935606809355063B
:10354000809154062091550630915606882309F043
:103550004AC0C901895097408F5A9440C8F40E94CC
:103560005C33615375478040904020F481E0809344
:1035700053060CC080915306882341F48091450680
:10358000882321F486E994E00E94BD0582E028C0EA
:1035900044E0203B340768F480914606882349F0D4
:1035A0001092530686E994E00E94BD0510924606EB
:1035B0007EC0205B34402955324008F078C08091AD
:1035C0004606813009F473C080914506882309F0CE
:1035D0006EC01092530686E994E00E94BD0581E01A
:1035E0008093460664C0215B344008F460C00E94AA
:1035F0005C33615375478040904008F041C0809132
:1036000053068823E9F5E0905706F090580600919C
:10361000590610915A0688EE93E0A0E0B0E0E80E5B
:10362000F91E0A1F1B1F0E945C33E616F7060807E7
:103630001907E8F581E08093530617C010925306EE
:1036400086E994E00E94BD0580914606823019F417
:103650001092460603C08F5F80934606809146060F
:10366000823018F082E0809346060E945C336093BB
:103670005706709358068093590690935A0617C0C0
:10368000E0905706F09058060091590610915A069E
:1036900088EE93E0A0E0B0E0E80EF91E0A1F1B1FC1
:1036A0000E945C33E616F7060807190738F21F91E7
:1036B0000F91FF90EF90089580915206843010F0A2
:1036C0000E94221A80915306882319F00E94461501
:1036D00008958091F90380FF08C060915F04809194
:1036E0005D0490E070E00E94B2188091460682303E
:1036F00008F0E8C1A82FB0E0FD01ED50FC4F80813B
:1037000085FF0BC0FD01E15FFB4F6081A35FBB4FF5
:103710008C9190E070E00E94B31480914606A82F2F
:10372000B0E0FD01ED50FC4F808186FF0BC0FD0134
:10373000ED5EFB4F6081AF5EBB4F8C9190E070E01F
:103740000E94741480914206882309F43FC080913E
:103750004606A82FB0E0FD01ED50FC4F808187FFA9
:103760000BC0FD01E95EFB4F6081AB5EBB4F8C91EE
:1037700090E070E00E94221480914606A82FB0E0ED
:10378000FD01EB50FC4F808184FF0BC0FD01E15D2A
:10379000FB4F6081A35DBB4F8C9190E070E00E9475
:1037A000C91380914606A82FB0E0FD01EB50FC4FF5
:1037B000808183FF0BC0FD01E55DFB4F6081A75D4C
:1037C000BB4F8C9190E070E00E94B2138091420652
:1037D000882309F483C08091D904823008F47EC024
:1037E00080914606A82FB0E0FD01E950FC4F808192
:1037F00087FF0BC0FD01E95BFB4F6081AB5BBB4FFB
:103800008C9190E070E00E94511380914606A82FA1
:10381000B0E0FD01E750FC4F808183FF0BC0FD014C
:10382000E959FB4F6081AB59BB4F8C9190E070E040
:103830000E945D1280914606A82FB0E0FD01E9507C
:10384000FC4F808182FF0BC0FD01ED5BFB4F60816F
:10385000AF5BBB4F8C9190E070E00E94FA128091B8
:103860004606A82FB0E0FD01E950FC4F808183FFA0
:103870000BC0FD01E55BFB4F6081A75BBB4F8C91EB
:1038800090E070E00E94A31280914606A82FB0E05D
:10389000FD01EB50FC4F808181FF0BC0FD01ED5D10
:1038A000FB4F6081AF5DBB4F8C9190E070E00E9458
:1038B0001B1280914606A82FB0E0FD01EB50FC4F93
:1038C000808180FF0BC0FD01E15EFB4F6081A35E44
:1038D000BB4F8C9190E070E00E94D9118091460618
:1038E000A82FB0E0FD01E750FC4F808186FF0BC0A0
:1038F000FD01E159FB4F6081A359BB4F8C9190E0D2
:1039000070E00E94991180914606A82FB0E0FD0159
:10391000ED50FC4F808182FF0BC0FD01E95FFB4F42
:103920006081AB5FBB4F8C9190E070E00E945911B9
:1039300080914606A82FB0E0FD01ED50FC4F80813C
:1039400081FF0BC0FD01ED5FFB4F6081AF5FBB4F9F
:103950008C9190E070E00E94191180914606A82F8A
:10396000B0E0FD01E950FC4F808184FF0BC0FD01F8
:10397000ED5AFB4F6081AF5ABB4F8C9190E070E0E5
:103980000E94D91080914606A82FB0E0FD01E950B1
:10399000FC4F808185FF0BC0FD01E95AFB4F608120
:1039A000AB5ABB4F8C9190E070E00E944110809127
:1039B0004606A82FB0E0FD01ED50FC4F808183FF4B
:1039C0000BC0FD01E55FFB4F6081A75FBB4F8C9192
:1039D00090E070E00E94FB0F80914606A82FB0E0B7
:1039E000FD01E950FC4F808180FF0BC0FD01E15CCF
:1039F000FB4F6081A35CBB4F8C9190E070E00E9414
:103A0000A60F80914606A82FB0E0FD01ED50FC4FB7
:103A1000808184FF0BC0FD01E55EFB4F6081A75EE6
:103A2000BB4F8C9190E070E00E94660F809146063B
:103A3000A82FB0E0FD01E550FC4F808181FF18C048
:103A400080913506FD01EB58FB4F813049F4A958B0
:103A5000BB4F6C91808190E070E00E947A0E08C0AC
:103A6000A958BB4F6C91808190E070E00E949D0E40
:103A700080914606A82FB0E0FD01EB50FC4F8081FD
:103A800087FF0BC0FD01E55CFB4F6081A75CBB4F6E
:103A90008C9190E070E00E94160E80914606A82F4F
:103AA000B0E0FD01E950FC4F808186FF0BC0FD01B5
:103AB000E55AFB4F6081A75ABB4F8C9190E070E0B4
:103AC0000E94BB0D089586E994E00E94BD050E9406
:103AD000ED140E94130A0895CF93DF93EC0186E959
:103AE00094E00E949404C817D9073CF086E994E05A
:103AF0000E948904892B09F42397CE01DF91CF918D
:103B00000895EF92FF920F931F93CF93DF9300914D
:103B1000460610E08AEF90E0089F7001099FF00CC4
:103B2000189FF00C1124C7010E94F80AF801ED500B
:103B3000FC4F882319F08081816002C080818E7FD4
:103B4000808380914606C82FD0E0C70102960E946C
:103B5000F80AC350DC4F888380914606C82FD0E016
:103B6000C70104960E94F80A90E00E946C1DC150A3
:103B7000DC4F88830091460610E0C70188569F4FAE
:103B80000E94F80AF801ED50FC4F882319F080815B
:103B9000806102C080818F7E808380914606C82F1D
:103BA000D0E0C70186569F4F0E94F80AC75EDB4FE0
:103BB000888380914606C82FD0E0C70184569F4F66
:103BC0000E94F80A90E00E946C1DC55EDB4F88835E
:103BD0000091460610E0C70106960E94F80AF80117
:103BE000ED50FC4F882319F08081826002C08081F3
:103BF0008D7F808380914606C82FD0E0C70108964C
:103C00000E94F80ACF5FDB4F888380914606C82F59
:103C1000D0E0C7010A960E94F80A90E00E946C1D4D
:103C2000CD5FDB4F88830091460610E0C7010C96FC
:103C30000E94F80AF801ED50FC4F882319F08081AA
:103C4000846002C080818B7F808380914606C82F6C
:103C5000D0E0C7010E960E94F80ACB5FDB4F888345
:103C600080914606C82FD0E0C70140960E94F80A0E
:103C700090E00E946C1DC95FDB4F8883009146066F
:103C800010E0C70142960E94F80AF801ED50FC4F7F
:103C9000882319F08081886002C08081877F8083BB
:103CA00080914606C82FD0E0C70144960E94F80ACA
:103CB000C75FDB4F888380914606C82FD0E0C701DD
:103CC00046960E94F80A90E00E946C1DC55FDB4F8B
:103CD00088830091460610E0C7014E960E94F80ABC
:103CE000F801ED50FC4F882319F08081806202C0FA
:103CF00080818F7D808380914606C82FD0E0C701E8
:103D000080960E94F80AC35FDB4F88838091460645
:103D1000C82FD0E0C70182960E94F80A90E00E9466
:103D20006C1DC15FDB4F88830091460610E0C70120
:103D300084960E94F80AF801ED50FC4F882319F090
:103D40008081806402C080818F7B80838091460661
:103D5000C82FD0E0C70186960E94F80ACF5EDB4FDD
:103D6000888380914606C82FD0E0C70188960E94BC
:103D7000F80A90E00E946C1DCD5EDB4F88830091B5
:103D8000460610E0C7018A960E94F80AF801ED5035
:103D9000FC4F882319F08081806802C080818F7772
:103DA000808380914606C82FD0E0C7018C960E9480
:103DB000F80ACB5EDB4F888380914606C82FD0E09F
:103DC000C7018E960E94F80A90E00E946C1DC95EA1
:103DD000DB4F88830091460610E0C701C0960E9421
:103DE000F80AF801EB50FC4F882319F080818160BC
:103DF00002C080818E7F808380914606C82FD0E0EC
:103E0000C701C2960E94F80AC35EDB4F8883809187
:103E10004606C82FD0E0C701C4960E94F80A90E079
:103E20000E946C1DC15EDB4F88830091460610E046
:103E3000C701C6960E94F80AF801EB50FC4F882390
:103E400019F08081826002C080818D7F80838091A3
:103E50004606C82FD0E0C701C8960E94F80ACF5D79
:103E6000DB4F888380914606C82FD0E0C701CA96F1
:103E70000E94F80A90E00E946C1DCD5DDB4F8883A4
:103E80000091460610E0C701CC960E94F80AF8019E
:103E9000EB50FC4F882319F08081846002C0808140
:103EA0008B7F808380914606C82FD0E0C701CE96D5
:103EB0000E94F80ACB5DDB4F888380914606C82FAD
:103EC000D0E0C701805C9F4F0E94F80A90E00E94FA
:103ED0006C1DC95DDB4F88830091460610E0C70169
:103EE000885B9F4F0E94F80AF801EB50FC4F882333
:103EF00019F08081806102C080818F7E80838091F3
:103F00004606C82FD0E0C701865B9F4F0E94F80A83
:103F1000C35DDB4F888380914606C82FD0E0C70180
:103F2000845B9F4F0E94F80A90E00E946C1DC15D67
:103F3000DB4F88830091460610E0C7018E5B9F4FE0
:103F40000E94F80AF801EB50FC4F882319F0808199
:103F5000886002C08081877F808380914606C82F59
:103F6000D0E0C7018C5B9F4F0E94F80AC75DDB4F12
:103F7000888380914606C82FD0E0C7018A5B9F4F97
:103F80000E94F80A90E00E946C1DC55DDB4F88839B
:103F90000091460610E0C701805B9F4F0E94F80A1F
:103FA000F801EB50FC4F882319F08081806202C039
:103FB00080818F7D808380914606C82FD0E0C70125
:103FC0008E5A9F4F0E94F80ACF5CDB4F8883809106
:103FD0004606C82FD0E0C7018C5A9F4F0E94F80AAE
:103FE00090E00E946C1DCD5CDB4F888300914606FB
:103FF00010E0C7018A5A9F4F0E94F80AF801EB505F
:10400000FC4F882319F08081806402C080818F7BFF
:10401000808380914606C82FD0E0C701885A9F4F01
:104020000E94F80ACB5CDB4F888380914606C82F3C
:10403000D0E0C701865A9F4F0E94F80A90E00E9484
:104040006C1DC95CDB4F88830091460610E0C701F8
:1040500082569F4F0E94F80AF801EB50FC4F8823CC
:1040600019F08081806802C080818F778083809181
:104070004606C82FD0E0C70180569F4F0E94F80A1D
:10408000C75CDB4F888380914606C82FD0E0C7010C
:104090008E559F4F0E94F80A90E00E946C1DC55CEF
:1040A000DB4F88830091460610E0C7018E599F4F71
:1040B0000E94F80AF801E950FC4F882319F080812A
:1040C000816002C080818E7F808380914606C82FE8
:1040D000D0E0C7018C599F4F0E94F80AC35CDB4FA8
:1040E000888380914606C82FD0E0C7018A599F4F28
:1040F0000E94F80A90E00E946C1DC15CDB4F88832F
:104100000091460610E0C70182599F4F0E94F80AAD
:10411000F801E950FC4F882319F08081846002C0C7
:1041200080818B7F808380914606C82FD0E0C701B5
:1041300080599F4F0E94F80ACF5BDB4F88838091A4
:104140004606C82FD0E0C7018E589F4F0E94F80A3C
:1041500090E00E946C1DCD5BDB4F8883009146068A
:1041600010E0C70184579F4F0E94F80AF801E950F8
:10417000FC4F882319F08081806802C080818F778E
:10418000808380914606C82FD0E0C70182579F4F99
:104190000E94F80ACB5BDB4F888380914606C82FCC
:1041A000D0E0C70180579F4F0E94F80A90E00E941C
:1041B0006C1DC95BDB4F88830091460610E0C70188
:1041C0008E569F4F0E94F80AF801E950FC4F882351
:1041D00019F08081826002C080818D7F8083809110
:1041E0004606C82FD0E0C7018C569F4F0E94F80AA0
:1041F000C35BDB4F888380914606C82FD0E0C701A0
:104200008A569F4F0E94F80A90E00E946C1DC15B85
:10421000DB4F88830091460610E0C7018C589F4F02
:104220000E94F80AF801E950FC4F882319F08081B8
:10423000886002C08081877F808380914606C82F76
:10424000D0E0C7018A589F4F0E94F80AC75BDB4F36
:10425000888380914606C82FD0E0C70188589F4FB9
:104260000E94F80A90E00E946C1DC55BDB4F8883BA
:104270000091460610E0C70186589F4F0E94F80A39
:10428000F801E950FC4F882319F08081806102C059
:1042900080818F7E808380914606C82FD0E0C70141
:1042A00084589F4F0E94F80ACF5ADB4F8883809131
:1042B0004606C82FD0E0C70182589F4F0E94F80AD7
:1042C00090E00E946C1DCD5ADB4F8883009146061A
:1042D00010E0C70180589F4F0E94F80AF801E9508A
:1042E000FC4F882319F08081806202C080818F7D1D
:1042F000808380914606C82FD0E0C7018E579F4F1C
:104300000E94F80ACB5ADB4F888380914606C82F5B
:10431000D0E0C7018C579F4F0E94F80A90E00E949E
:104320006C1DC95ADB4F88830091460610E0C70117
:104330008A579F4F0E94F80AF801E950FC4F8823E2
:1043400019F08081806402C080818F7B808380919E
:104350004606C82FD0E0C70188579F4F0E94F80A31
:10436000C75ADB4F888380914606C82FD0E0C7012B
:1043700086579F4F0E94F80A90E00E946C1DC55A14
:10438000DB4F88830091460610E0C7018C559F4F94
:104390000E94F80AF801E750FC4F882319F0808149
:1043A000816002C080818E7F808380914606C82F05
:1043B000D0E0C7018A559F4F0E94F80AC35ADB4FCD
:1043C000888380914606C82FD0E0C70188559F4F4B
:1043D0000E94F80A90E00E946C1DC15ADB4F88834E
:1043E0000091460610E0C70180559F4F0E94F80AD1
:1043F000F801E750FC4F882319F08081846002C0E7
:1044000080818B7F808380914606C82FD0E0C701D2
:104410008E549F4F0E94F80ACF59DB4F88838091BA
:104420004606C82FD0E0C7018C549F4F0E94F80A5F
:1044300090E00E946C1DCD59DB4F888300914606A9
:1044400010E0C7018A549F4F0E94F80AF801E75014
:10445000FC4F882319F08081886002C08081877FAB
:10446000808380914606C82FD0E0C70188549F4FB3
:104470000E94F80ACB59DB4F888380914606C82FEB
:10448000D0E0C70186549F4F0E94F80A90E00E9436
:104490006C1DC959DB4F88830091460610E0C701A7
:1044A00084549F4F0E94F80AF801E750FC4F88237C
:1044B00019F08081806102C080818F7E808380912D
:1044C0004606C82FD0E0C70182549F4F0E94F80AC9
:1044D000C759DB4F888380914606C82FD0E0C701BB
:1044E00080549F4F0E94F80A90E00E946C1DC559AD
:1044F000DB4F88830091460610E0C701845A9F4F26
:104500000E94F80AF801E750FC4F882319F08081D7
:10451000806402C080818F7B808380914606C82F93
:10452000D0E0C701825A9F4F0E94F80AC359DB4F5F
:10453000888380914606C82FD0E0C701805A9F4FDC
:104540000E94F80A90E00E946C1DC159DB4F8883DD
:104550000091460610E0C70180529F4F0E94F80A62
:10456000F801E550FC4F882319F08081846002C077
:1045700080818B7F808380914606C82FD0E0C70161
:104580008E519F4F0E94F80ACF58DB4F888380914D
:104590004606C82FD0E0C7018C519F4F0E94F80AF1
:1045A00090E00E946C1DCD58DB4F88830091460639
:1045B00010E0C7018C529F4F0E94F80AF801E550A5
:1045C000FC4F882319F08081826002C080818D7F3A
:1045D000808380914606C82FD0E0C7018A529F4F42
:1045E0000E94F80ACB58DB4F888380914606C82F7B
:1045F000D0E0C70188529F4F0E94F80A90E00E94C5
:104600006C1DC958DB4F8883DF91CF911F910F91AB
:10461000FF90EF9008954F925F927F928F929F92BA
:10462000AF92BF92CF92DF92EF92FF920F931F93C0
:10463000DF93CF93CDB7DEB7C854D0400FB6F89410
:10464000DEBF0FBECDBF06E914E0C8010E94BD0564
:10465000C80166E049E00E949804C8010E94700504
:1046600000D000D0EDB7FEB71283018381E592E060
:10467000948383830E94B22B0F900F900F900F9022
:10468000C8010E94540500D000D009E714E0EDB73E
:10469000FEB71283018381E492E0948383830E94B6
:1046A000B22B46E3442E42E0542EEE24FF24CC24C9
:1046B000DD240F900F900F900F90702E012F39E096
:1046C000A32EB12CAC0EBD1E4E010894811C911C72
:1046D00089E794E00E94662C982F8D3031F08D3060
:1046E000DCF180538230C0F530C01830A1F59981DB
:1046F000892F8053823078F5913311F490E801C00E
:1047000090E08A81813309F4905C8B81813309F4D4
:10471000905E8C81813309F4905F8D81813309F43F
:10472000985F8E81813309F49C5F8F81813309F416
:104730009E5F8885813309F49F5FF501EE0DFF1DB3
:1047400090830894E11CF11C06C0F401E10FF11DF7
:1047500090831F5F01C010E0F0E4EF16F104C9F48C
:1047600086E994E0B601A5010E94A8040894C11C42
:10477000D11C00D000D0EDB7FEB771820283548205
:1047800043820E94B22BEE24FF240F900F900F90D3
:104790000F90FFEFCF16D10409F00CF499CFC85B4E
:1047A000DF4F0FB6F894DEBF0FBECDBFCF91DF91C4
:1047B0001F910F91FF90EF90DF90CF90BF90AF903F
:1047C0009F908F907F905F904F900895BF92CF926F
:1047D000DF92EF92FF920F931F93DF93CF93CDB7AA
:1047E000DEB72E970FB6F894DEBF0FBECDBF73E0D5
:1047F000B72E67E0E62EF12CEC0EFD1E53E0C52E21
:10480000D12CCC0EDD1E30C30E945C3360527E443E
:1048100080409040C8F40E945C33695873418040E6
:10482000904090F01A3011F01D3031F48091FD0568
:104830008F5F8093FD0502C01092FD058091FD05FC
:10484000833011F40E940B23812F63EF74E00E94E8
:104850001A07882311F400E001C38091F7049091B6
:10486000F804A091F904B091FA048A3B47EC94074C
:1048700041E2A40744E7B40709F41EC18B3B57EC9F
:10488000950751E2A50754E7B50708F086C08E3CAE
:10489000E8E49E07E7E5AE07EAE1BE0709F4DFC1F9
:1048A0008F3CF8E49F07F7E5AF07FAE1BF0708F090
:1048B0003AC084302AE9920727EDA2072EE0B2071A
:1048C00009F46DC185303AE9930737EDA3073EE05F
:1048D000B30780F486314AEA940747E3A4074BE024
:1048E000B40709F45CC184559447A54CBB4009F05A
:1048F000ABC241C28839ECE29E07EAE1AE07E6E1CD
:10490000BE0709F455C18035FFED9F07FDEEAF07E7
:10491000F8E1BF0709F44FC28259934AAC4EB44143
:1049200009F092C23CC188323EE5930732EDA307FD
:1049300034E2B30709F433C189324EE5940742EDFE
:10494000A40744E2B40780F484375BEE95075AE786
:10495000A5075BE1B50709F422C1825D924CA2482C
:10496000BE4109F071C224C1863EF5ED9F07FAED04
:10497000AF07F3E3BF0709F49FC080362BED920722
:104980002BE3A2072EE6B20709F409C18E57994A14
:10499000AB45B64209F058C20BC18E3F46EB9407B7
:1049A00049E2A40745EAB40709F459C18F3F56EB21
:1049B000950759E2A50755EAB50708F03AC08235D0
:1049C000EAEE9E07E0E8AE07EAE8BE0709F4E7C0B2
:1049D0008335FAEE9F07F0E8AF07FAE8BF0780F4E7
:1049E000863E26EA920726E2A2072DE7B20709F4DF
:1049F00036C180589C4DA544B24809F025C2BBC1C0
:104A00008E3742E194074AE6A4074BE9B40709F45C
:104A1000C6C08A3756EF950751EFA5075DE9B50780
:104A200009F41DC18C589548A74AB84909F00CC231
:104A300016C18436F9ED9F07F0EEAF07F7EDBF071B
:104A400009F43AC0853629ED920720EEA20727ED3A
:104A5000B207C8F4803834E7930730E1A30734EC99
:104A6000B30709F4A5C084354DE294074FEFA407BE
:104A700045ECB40709F493C08A58974FA74CB84B3C
:104A800009F0E2C195C08E34EDE59E07EEE3AE0776
:104A9000E3EEBE0709F483C0823FFDEE9F07F4E218
:104AA000AF07FDEFBF0709F481C1865B9342A34ABC
:104AB000B24E09F0C9C1D3C00E945C336093BA04FE
:104AC0007093BB048093BC049093BD04B092B9046E
:104AD00080910D0590910E05A0910F05B0911005E4
:104AE000F70180839183A283B3836F817885898561
:104AF0009A850E9489367093BF046093BE048091AA
:104B0000110590911205A0911305B0911405F701BC
:104B100080839183A283B3836F81788589859A8509
:104B20000E9489367093C1046093C004809115057A
:104B300090911605A0911705B0911805F701808393
:104B40009183A283B3836F81788589859A850E943A
:104B500089368B017093C3046093C2046091C404CE
:104B60007091C5048091C6049091C70420E030E0A4
:104B700040E050E00E941A36882379F4B801882773
:104B800077FD8095982F0E94BC366093C80470937F
:104B9000C9048093CA049093CB0401E056C180916C
:104BA000FD048093CC048091FE048093CD044CC11D
:104BB0008091FD049091FE04A091FF04B091000546
:104BC000F70180839183A283B3836F817885898580
:104BD0009A8520E030E048EC52E40E94EF370E94D2
:104BE00089367093CF046093CE04693C710520F040
:104BF0001092CF041092CE04809117059091180561
:104C00009093D1048093D0048091190590911A0556
:104C10009093D3048093D20480911D0590911E053A
:104C200090939102809390028091210590912205AA
:104C30009093930280939202809123059091240592
:104C4000909395028093940280912505909126057A
:104C50009A8389839093970280939602F5C060911E
:104C6000FD047091FE048091FF04909100050E9464
:104C7000BC3620E836E948E15BE40E9421366093C7
:104C8000C4047093C5048093C6049093C7046091D4
:104C90000105709102058091030590910405D601EC
:104CA0006C9311967C93119712968C93129713968E
:104CB0009C930E94BC3620E836E948E15BE40E9400
:104CC00021366093D4047093D5048093D6049093D6
:104CD000D704809122058093D80480912105809388
:104CE000D90480910D0590910E05A0910F05B0910A
:104CF0001005F70180839183A283B3838F81988508
:104D0000A985BA858093C8049093C904A093CA0466
:104D1000B093CB048091050590910605A0910705FD
:104D2000B091080580839183A283B3838F81988596
:104D3000A985BA858093DA049093DB04A093DC0400
:104D4000B093DD048091110590911205A091130597
:104D5000B091140580839183A283B3838F8198855A
:104D6000A985BA858093DE049093DF04A093E004C4
:104D7000B093E10469C08091050590910605A0916A
:104D80000705B0910805F70180839183A283B3835F
:104D90008F819885A985BA85B0588093E204909355
:104DA000E304A093E404B093E5044EC08091FD04B5
:104DB0008093E60449C08091FD049091FE04A09187
:104DC000FF04B0910005F70180839183A283B38330
:104DD0008F819885A985BA858093E7049093E8042C
:104DE000A093E904B093EA04809101059091020533
:104DF000A0910305B091040580839183A283B383BE
:104E00008F819885A985BA858093EB049093EC04F3
:104E1000A093ED04B093EE048091050590910605F2
:104E2000A0910705B091080580839183A283B38385
:104E30008F819885A985BA858093EF049093F004BB
:104E4000A093F104B093F20400E08091F404823264
:104E500029F483EF94E063E20E94EA098EEB90E08C
:104E60000E94C333002341F589E794E00E94362C69
:104E70001816190604F589E794E00E94662C182F8D
:104E80008091B904882309F0DFCCBECC1092B9041C
:104E900001E0802F90E02E960FB6F894DEBF0FBE93
:104EA000CDBFCF91DF911F910F91FF90EF90DF90D9
:104EB000CF90BF90089500E02091BA043091BB04D8
:104EC0004091BC045091BD04205F384D4F4F5F4F5F
:104ED0002B873C874D875E870E945C332B853C8502
:104EE0004D855E85261737074807590778F2D1CFD9
:104EF0006F927F928F929F92AF92BF92CF92DF92EA
:104F0000EF92FF920F931F93E0906106F09062067C
:104F100000916306109164068FE590E0A0E0B0E098
:104F2000E80EF91E0A1F1B1F0E945C336E157F05D9
:104F30008007910708F427C10E945C333B014C01B4
:104F4000A0906106B0906206C0906306D09064069F
:104F50000E945C33609361067093620680936306DF
:104F60009093640680E00E94F834AA2797FDA095EC
:104F7000BA2FBC01CD010E94BC362DEC3CEC4CE8B4
:104F80005FE30E94EF3720E030E040E85AE30E9400
:104F9000EF377B018C0160913706709138068827C6
:104FA00077FD8095982F0E94BC3620E030E048ECD9
:104FB00052E40E9421369B01AC01C801B7010E9456
:104FC000EF372DEC3CEC4CE45EE30E94EF377B01C5
:104FD0008C0160919C0270919D0280919E02909143
:104FE0009F022DEC3CEC4CE45FE30E94EF379B0109
:104FF000AC01C801B7010E945435DC019B01AC0132
:1050000020939C0230939D0240939E0250939F02F6
:10501000CB018093160690931706A0931806B093C1
:10502000190680913B0690913C06181619060CF063
:10503000AAC081E00E94F834AA2797FDA095BA2F54
:10504000BC01CD010E94BC362DEC3CEC4CE85FE38A
:105050000E94EF3720E030E040E85AE30E94EF374B
:105060007B018C016091390670913A06882777FDA3
:105070008095982F0E94BC3620E030E44CE156EC3D
:105080000E9421369B01AC01C801B7010E94543532
:105090007B018C0160913B0670913C06882777FD6F
:1050A0008095982F0E94BC3620E030E048EC52E416
:1050B0000E9421369B01AC01C801B7010E94EF3765
:1050C0002DEC3CEC4CE45EE30E94EF377B018C015D
:1050D0006091690670916A0680916B0690916C06EA
:1050E0002DEC3CEC4CE45FE30E94EF379B01AC01FC
:1050F000C801B7010E9454357B018C016093690699
:1051000070936A0680936B0690936C06B3016A19DC
:105110007B0980E090E00E94BA369B01AC01C80197
:10512000B7010E94EF372FEA35EA41E959E30E94BF
:10513000EF372091650630916606409167065091E1
:1051400068060E9454355B016C016093650670939C
:1051500066068093670690936806C801B70120E051
:1051600030E048EC52E40E94EF370E948936709399
:10517000150660931406C601B5010E948E36709321
:105180001306609312061F910F91FF90EF90DF902E
:10519000CF90BF90AF909F908F907F906F90089529
:1051A000EF92FF920F931F9380914406882351F052
:1051B00083E00E94F83464E070E00E941539609347
:1051C00002063CC083E00E94F834AA2797FDA09510
:1051D000BA2FBC01CD010E94BC362DEC3CEC4CE456
:1051E0005EE30E94EF3720E030E040E85EE30E949B
:1051F000EF377B018C016091020670E0882777FD14
:105200008095982F0E94BC362DEC3CEC4CE45FE37B
:105210000E94EF379B01AC01C801B7010E945435D1
:105220000E948E3620915F06621730F030915E0644
:10523000262F361708F4232F209302061F910F9173
:10524000FF90EF90089583E00E94F534089583E085
:105250000E94F53408951F93CF93DF9385E090E08B
:105260006CE070E00E94231568EE73E080E090E04F
:105270000E946A3389E794E00E94B32CC0E0D0E03A
:1052800010E0CE016DE171E00E941539892BA9F47F
:105290001F5E86E994E0612F4CE00E94980486E945
:1052A00094E00E94700586E994E06EEE0E94A005ED
:1052B00086E994E00E945405105161E070E080E0BE
:1052C00090E00E946A33219687E0C13DD807C9F675
:1052D000DF91CF911F91089586E061E00E94A13493
:1052E00008950F931F9386E061E00E94623409E7FE
:1052F00014E0C80140E051EE60E070E00E94D42B61
:1053000010939106009390060E946C2986E994E020
:105310000E94F6050E94631D64EF71E080E090E05A
:105320000E946A3383EF93E00E94F80A813011F003
:105330000E94090D0E94690A1092460607C00E9449
:10534000811D809146068F5F8093460680914606B8
:105350008230A8F3109246060E942B290E9423292E
:105360000E94272988EA94E064E47BE224E630E0A6
:1053700040E050E000E00E94873286E994E00E941D
:10538000BD0588EA94E00E94ED321F910F910895C7
:105390002F923F924F925F926F927F928F929F9245
:1053A000AF92BF92CF92DF92EF92FF920F931F9333
:1053B000DF93CF9300D000D0CDB7DEB78091420607
:1053C000882309F4E1C0E0906D06F0906E0600912C
:1053D0006F0610917006C801B7019F7725E33AEF79
:1053E0004EE85CE30E94EF370E941E3669837A83A1
:1053F0008B839C83C801B7012091C4043091C504FC
:105400004091C6045091C7040E9453351B012C01E2
:105410009F7720EC3BE649ED57E40E94EF375B01B4
:105420006C01609171067091720680917306909183
:1054300074062091D4043091D5044091D604509143
:10544000D7040E9453353B014C019F7720EC3BE68B
:1054500049ED57E40E94EF3729813A814B815C8105
:105460000E94EF377B018C01C601B501A6019501B1
:105470000E94EF375B016C01C801B701A8019701D9
:105480000E94EF379B01AC01C601B5010E94543563
:105490000E9476380E94893660932F0670933006FA
:1054A000809331069093320660E070E080E89FE3DD
:1054B00029813A814B815C810E9421369B01AC019C
:1054C000C201B1010E94EF3797FA909497F8909437
:1054D000A40193010E94C73520EE3EE245E652E466
:1054E0000E94EF3720E030E044EB52E40E94543554
:1054F0000E9489369B01AC0197FF04C028593E4F9A
:105500004F4F5F4FCA01B901645B704080409040CB
:1055100097FF06C0CA01B9016C547F4F8F4F9F4F50
:105520000E94BC362091C8043091C9044091CA043D
:105530005091CB040E9453350E94893697FF04C0D6
:1055400068597E4F8F4F9F4F0E94BC3620E030E05D
:1055500044EB53E40E94213620E030E040E851E47F
:105560000E94EF370E94523820E030E040E85FE3CD
:105570000E9454350E948E3660932E06613108F4E5
:105580006CC010922E0669C08091D904823008F454
:1055900064C08091D804853008F45FC0A09075067F
:1055A0008DE18A1508F459C0E090DA04F090DB042C
:1055B0000091DC041091DD0460917606709177060D
:1055C0008091780690917906A80197010E94533541
:1055D0009F7720E030E040E05FE30E94E437181658
:1055E0005CF410927506E0927606F09277060093CE
:1055F00078061093790631C08A2D8F5F80937506E7
:105600008E3159F58091C4049091C504A091C604CF
:10561000B091C70480936D0690936E06A0936F06B9
:10562000B09370068091D4049091D504A091D604D3
:10563000B091D7048093710690937206A09373067D
:10564000B0937406E0922A06F0922B0600932C0683
:1056500010932D0681E0809342060F900F900F90DB
:105660000F90CF91DF911F910F91FF90EF90DF90FE
:10567000CF90BF90AF909F908F907F906F905F90F2
:105680004F903F902F900895CF92DF92EF92FF922C
:105690000F931F930E9478270E94D02880910206C2
:1056A000282F30E03093990220939802809144068D
:1056B000882359F500915F0610E0201B310BB901DA
:1056C000882777FD8095982F0E94BC366B017C015E
:1056D00060915E0670E0601B710B882777FD8095F6
:1056E000982F0E94BC369B01AC01C701B6010E94F5
:1056F000213620E030E048EC52E40E94EF370E946F
:1057000089367093990260939802809198029091E3
:1057100099028D599F4F34F48DE99FEF9093990230
:10572000809398020E9477080E94FE0A86E994E01E
:105730000E94C8290E945C1B1F910F91FF90EF905F
:10574000DF90CF9008950E94E623892B19F00E94E4
:10575000442B089588EA94E00E94D53208958FEF93
:105760009FE70895DF93CF93CDB7DEB7FE0139965B
:105770008D819E8161E04F8158859F010E94532E4B
:10578000CF91DF910895DF93CF93CDB7DEB7FE01C0
:1057900039968D819E8160E04F8158859F010E94DE
:1057A000532ECF91DF9108950F931F93DC01ED915C
:1057B000FC910288F389E02D20E030E000E010E069
:1057C00009951F910F9108958F92AF92CF92EF920A
:1057D000FF920F931F93DF93CF93CDB7DEB7FC01FA
:1057E0001382128288EE93E0A0E0B0E08483958378
:1057F000A683B7838BED93E091838083558744879D
:1058000037872687118B008BF38AE28AC48AA58AA0
:10581000868A70E0CB0123E0880F991F2A95E1F773
:105820009C012258394F308F278B8A57994F928F7E
:10583000818F81E090E002C0880F991F6A95E2F79E
:1058400020918E06282B20938E06CF0140E051EE4A
:1058500060E070E00E94D42BCF91DF911F910F91F7
:10586000FF90EF90CF90AF908F900895FC01838DC3
:10587000882319F42FEF3FEF0DC00788F08DE02D3E
:105880002081318182819381281B390B848195810C
:1058900028233923C9010895FC01838D882319F435
:1058A0002FEF3FEF11C0018CF28DE02D208131816F
:1058B00082819381281B390B2095309584819581B5
:1058C000282339232F5F3F4FC9010895FC01838DA1
:1058D000882361F0A789B08D2D913C911197129684
:1058E0008D919C9113972817390721F44FEF5FEFA3
:1058F000CA01089512968D919C9113971696ED9179
:10590000FC911797E80FF91F408112968D919C9199
:105910001397019614962D913C911597822393230A
:1059200013969C938E93129750E0E2CFFC01838DE7
:10593000882351F00788F08DE02D2081318182810C
:1059400093812817390721F42FEF3FEFC9010895FC
:10595000828193810680F781E02DE80FF91F808115
:10596000282F30E0F3CFDC015796ED91FC9158974A
:1059700082819381918380835996ED91FC915A970E
:1059800080819181938382830895DC015B968C9161
:105990005B978823A9F15996ED91FC915A97208144
:1059A00031812F5F3F4F84819581282339235C9675
:1059B0008C915C97882329F082819381281739077D
:1059C000F9F08281938128173907D9F38081918179
:1059D0000680F781E02DE80FF91F60835996ED915D
:1059E000FC915A97318320835296ED91FC91539705
:1059F000808156969C91892B808321E030E002C003
:105A000020E030E0C9010895CF93DF93EC011B82C1
:105A10001A828A819B81998388831D821C828E8150
:105A20009F81009721F00E94EA031F821E82DF916E
:105A3000CF9108950F931F938C01DC015296ED9145
:105A4000FC915397208156968C91569755969C9130
:105A50005597892B80958223808357968D919C91B1
:105A600058970E94042DF801818D928D0E94042D7B
:105A7000D8015B961C921F910F9108950F931F936D
:105A8000CF93DF938C01FC01138212828281938178
:105A90009183808341E0A1E0B0E001C04F5FFD0150
:105AA000042E02C0EE0FFF1F0A94E2F79B0182E072
:105AB0006130780710F020E032E0E217F30770F36E
:105AC000C1E0D0E002C0CC0FDD1F4A95E2F721977C
:105AD000F801268137812115310541F084819581B6
:105AE0008C179D0789F0C9010E94EA03F801D5834C
:105AF000C483CE0101960E9440039C01F801978364
:105B0000868380E0232B09F081E0DF91CF911F9104
:105B10000F910895AF92BF92CF92DF92EF92FF92D2
:105B20000F931F93CF93DF937C015A016B01E9011F
:105B3000DC015B968C915B978823F1F02115310590
:105B400039F45796ED91FC915897C481D5812196EF
:105B50000115110549F4D7015996ED91FC915A9719
:105B6000048115810F5F1F4FD701ED91FC910088D3
:105B7000F189E02DC7010995F7018789908D20975C
:105B800011F4C0E8D0E0BE010E943E2D882381F0D0
:105B9000D70159968D919C915A970115110511F4D1
:105BA00000E110E0B8010E943E2D882309F04DC0AD
:105BB000D701ED91FC910088F189E02DC70109958D
:105BC00067C0D7015096ED91FC915197B0E0AB16AC
:105BD000B1EEBB06B0E0CB06B0E0DB0609F454C082
:105BE00081E090E0D70154960C9002C0880F991F75
:105BF0000A94E2F7808360E079E08DE390E0A6010B
:105C000095010E944A392150304040405040CA011D
:105C1000B90122E030E040E050E00E944A39D7016B
:105C20001C96ED91FC911D9730831E96ED91FC9191
:105C30001F972083D7015296ED91FC915397808155
:105C400055969C91892B808323C0D7015996ED915D
:105C5000FC915A971382128282819381918380836F
:105C60005796ED91FC91589713821282828193810D
:105C70009183808381E05B968C931A141B041C042F
:105C80001D040CF49ECFD6CF108220E130E0C7CFA8
:105C9000DF91CF911F910F91FF90EF90DF90CF9008
:105CA000BF90AF9008952F923F924F925F926F9264
:105CB0007F928F929F92AF92BF92CF92DF92EF929C
:105CC000FF920F931F93DF93CF93CDB7DEB7649707
:105CD0000FB6F894DEBF0FBECDBF3C01688B5A8B68
:105CE000498B69011C01AE014F5F5F4F5C8B4B8B91
:105CF000E989FA89488940FD659140FF6191FA8BF5
:105D0000E98B662309F4D7C3653249F440FD8591D8
:105D100040FF8191FA8BE98B8532B1F40CC06A3077
:105D200051F4D301ED91FC910190F081E02DC1017E
:105D30006DE009956AE0D301ED91FC910190F0814D
:105D4000E02DC1010995D4CF982F10E08824992423
:105D50001032B0F49B3269F09C3228F4903251F04A
:105D6000933271F40BC09D3239F0903349F41160D5
:105D700028C01260146025C0186023C0106121C0C3
:105D800017FD2BC0892F80538A3078F416FF06C088
:105D9000BAE09B9E902C1124980E13C0EAE08E9ED0
:105DA000802C1124880E10620CC09E3221F416FD46
:105DB00082C3106406C09C3611F4106802C0983685
:105DC00061F4E989FA89488940FD959140FF9191F4
:105DD000FA8BE98B992309F0BBCF892F8554833047
:105DE00020F4812F8061905E07C0892F8556833013
:105DF00008F0E6C1812F8F7E86FD02C076E0972EE7
:105E00006FE3F62EF822953619F450E4F52A07C010
:105E1000963619F480E8F82A02C091109A94F7FE99
:105E20000BC09BE3991520F427E05CE3B52E0DC071
:105E3000B92CB39427E009C0A7E0A91520F447E0E6
:105E4000942E27E001C0292DBB24F6013496FD874E
:105E5000EC87D6016D917D918D919C91AE014F5F44
:105E60005F4F0B2D0E9468026C010981E02FF0E06A
:105E7000FF87EE8700FF05C0FE85F3FD02C01DE22F
:105E800009C0F1FE02C01BE205C0F2FC02C010E036
:105E900001C010E28E859F858C709070892B09F46B
:105EA00044C0112311F483E001C084E0881510F090
:105EB00088240EC0881AF3FC0BC0D301ED91FC912D
:105EC0000190F081E02DC10160E209958A94A9F763
:105ED000112349F0D301ED91FC910190F081E02D67
:105EE000C101612F0995BE85B3FF03C00AE513E028
:105EF00012C00EE513E00FC0E114F10409F0605286
:105F0000D301ED91FC910190F081E02DC101099543
:105F10000F5F1F4F05C0EF2CFF24B0E1EB22FF24E1
:105F2000F8016491662341F748C1F7FE13C0BC0C29
:105F3000FE85F4FF04C08A81813309F4BA941B14EE
:105F40001CF0BB24B3942DC048E04B1550F538E04D
:105F5000B32E27C0F6FC25C0892D90E08C159D0539
:105F60004CF05CEFC5165FEFD50624F080E8F82A08
:105F700001C09A94992049F0E2E0F0E0EC0FFD1F97
:105F8000E90DF11D80818033A1F3F7FE0AC0B92C21
:105F9000B394892D90E0C816D90614F0992401C055
:105FA0009C18F7FC03C025E030E009C01C141D0458
:105FB0001CF021E030E003C096012F5F3F4F11231A
:105FC00011F02F5F3F4F992029F0892D90E0019625
:105FD000280F391F882D90E02817390714F08824DE
:105FE00001C0821A4F2C5524C20189709070892BF0
:105FF00059F00CC0D301ED91FC910190F081E02D9E
:10600000C10160E209958A948820A1F7112349F023
:10601000D301ED91FC910190F081E02DC101612F40
:10602000099543FE0BC00CC0D301ED91FC9101908A
:10603000F081E02DC10160E309958A948820A1F7E1
:10604000F7FE51C08601D7FE02C000E010E07601E5
:106050000894E11CF11CE01AF10AE1E0F0E0EC0F19
:10606000FD1FEE0EFF1E26014B185108892D90E0F2
:10607000AA24BB24A81AB90AFFEF0F3F1F0749F44F
:10608000D301ED91FC910190F081E02DC1016EE210
:106090000995C016D10634F0401651061CF4F701DC
:1060A000608101C060E3015010400894E11CF11CC4
:1060B0000A151B054CF0D301ED91FC910190F08184
:1060C000E02DC1010995D8CF0C151D0541F48A8139
:1060D000863320F4853319F4BE85B4FF61E3D30120
:1060E000ED91FC9165C06A81613309F00F7ED301A7
:1060F000ED91FC910190F081E02DC101099599206D
:10610000E1F0D301ED91FC910190F081E02DC1010E
:106110006EE2099512E0E1E0F0E0EC0FFD1FE10F07
:10612000F11D60811F5FD301ED91FC910190F08121
:10613000E02DC10109959A9471F7D301ED91FC917D
:106140000190F081E02D44FC02C065E601C065E4E9
:10615000C1010995D7FC05C0C114D10441F404FF65
:1061600006C0D094C194D108D3946DE201C06BE213
:10617000D301ED91FC910190F081E02DC1010995D1
:1061800060E305C06F5FE6EFFFEFCE0EDF1EFAE0C3
:10619000CF16D104BCF7D301ED91FC910190F081B1
:1061A000E02DC1010995D301ED91FC916C2D605D4D
:1061B0000190F081E02DC1010995CC84DD8478C186
:1061C000933631F0933799F0933509F061C023C0CD
:1061D000F601808189835E010894A11CB11C42E014
:1061E00050E0C40ED51E21E0E22EF12C12C0D601E3
:1061F000AD90BC9016FD03C06FEF7FEF02C0692D1C
:1062000070E0E2E0F0E0CE0EDF1EC5010E944D041A
:106210007C011F7713C0D601AD90BC9016FD03C062
:106220006FEF7FEF02C0692D70E0E2E0F0E0CE0E8C
:10623000DF1EC5010E9442047C01106813FF0BC0E1
:1062400023C0D301ED91FC910190F081E02DC101BB
:1062500060E209958A94882D90E0E816F90688F3A3
:1062600013C0F50117FD659117FF61915F01D3011F
:10627000ED91FC910190F081E02DC1010995811013
:106280008A940894E108F108E114F10451F710C16F
:10629000943611F0993699F517FF0AC0F60120815E
:1062A00031814281538184E090E0C80ED91E0CC038
:1062B000D6018D919C919C01442737FD4095542F28
:1062C000E2E0F0E0CE0EDF1E9FE6F92EF12257FF4E
:1062D00009C050954095309521953F4F4F4F5F4FE6
:1062E000F0E8FF2ACA01B901AE014F5F5F4F2AE013
:1062F00030E00E940A02E82E4B89E41A41C095372B
:1063000021F41F7E2AE030E01CC0197F9F3661F027
:10631000903720F4983509F0CEC00FC0903739F08F
:10632000983709F0C8C004C028E030E00AC0106106
:1063300014FD146020E130E004C014FD166020E17B
:1063400032E017FF08C0D6016D917D918D919C912F
:10635000E4E0F0E008C0D6018D919C91BC0180E0A2
:1063600090E0E2E0F0E0CE0EDF1EAE014F5F5F4F47
:106370000E940A02E82EFB89EF1A8FE7F82EF1221D
:10638000F6FE0BC04EEFF422E91438F4F4FE07C019
:10639000F2FC05C05FEEF52202C01E2D01C0192DD2
:1063A000F4FE0DC0FE01EE0DF11D8081803319F465
:1063B00089EEF82208C01F5FF2FE05C003C08F2DD2
:1063C000867809F01F5F0F2DF3FC18C0F0FE13C094
:1063D000181510F09E2C0FC09E2C980C911A182D99
:1063E0000AC0D301ED91FC910190F081E02DC10133
:1063F00060E209951F5F1815A0F304C0181510F48A
:10640000811A01C0882404FF17C0D301ED91FC91CB
:106410000190F081E02DC10160E3099502FF29C0E0
:10642000D301ED91FC910190F081E02D01FD02C0BE
:1064300068E712C068E510C0802F8678D1F001FFB0
:1064400002C06BE201C060E2F7FC6DE2D301ED91A6
:10645000FC910190F081E02DC10109950AC0D301A2
:10646000ED91FC910190F081E02DC10160E309956F
:106470009A94E914A0F3EA94D301ED91FC91A1E080
:10648000B0E0AC0FBD1FAE0DB11D0190F081E02D4D
:10649000C1016C910995EE2071F70AC0D301ED910D
:1064A000FC910190F081E02DC10160E209958A9490
:1064B0008820A1F71DCC64960FB6F894DEBF0FBEFE
:1064C000CDBFCF91DF911F910F91FF90EF90DF90A3
:1064D000CF90BF90AF909F908F907F906F905F9084
:1064E0004F903F902F900895F999FECF72BD61BDF6
:1064F000F89A80B50895F999FECF1FBA72BD61BDB3
:1065000040BD0FB6F894FA9AF99A0FBE08950F930A
:10651000FC016115710511F480E011C02183328303
:1065200043835483728761870170000F000F000F4F
:106530008081877F802B82608B7F808381E00F91B9
:106540000895CF93DF93EC010E945C339B01AC0173
:106550008D819E81AF81B885281739074A075B076F
:1065600028F4888184FD02C060E00DC089819A8191
:10657000AB81BC81820F931FA41FB51F8D839E83A7
:10658000AF83B88761E0222757FD2395332744273F
:106590005527922F91709295907F88818F7E892BBD
:1065A0008883862FDF91CF910895CF93DF93EC01FD
:1065B000888182FF0FC0CE010E94A132882351F052
:1065C000E985FA85309709F00995888183FF02C033
:1065D0008B7F8883DF91CF910895CF93DF93EC0178
:1065E00089859A85892BE1F089819A81AB81BC816B
:1065F0000097A105B105A1F00E945C3329813A8181
:106600004B815C81260F371F481F591F2D833E8306
:106610004F835887888184608F7E888381E001C0A2
:1066200080E0DF91CF9108951F920F920FB60F92E5
:1066300011242F933F938F939F93AF93BF93809198
:10664000960690919706A0919806B0919906309180
:106650009A060196A11DB11D232F2D5F2D3720F025
:106660002D570196A11DB11D20939A068093960681
:1066700090939706A0939806B093990680919206FE
:1066800090919306A0919406B09195060196A11D54
:10669000B11D8093920690939306A0939406B093B5
:1066A0009506BF91AF919F918F913F912F910F9040
:1066B0000FBE0F901F9018958FB7F89420919606F3
:1066C0003091970640919806509199068FBFB90175
:1066D000CA0108959B01AC017FB7F894809192069E
:1066E00090919306A0919406B091950666B5A89BEB
:1066F00005C06F3F19F00196A11DB11D7FBFBA2FD4
:10670000A92F982F8827860F911DA11DB11D62E02A
:10671000880F991FAA1FBB1F6A95D1F7BC012DC016
:10672000FFB7F8948091920690919306A0919406F9
:10673000B0919506E6B5A89B05C0EF3F19F001960C
:10674000A11DB11DFFBFBA2FA92F982F88278E0F2B
:10675000911DA11DB11DE2E0880F991FAA1FBB1F4B
:10676000EA95D1F7861B970B885E9340C8F22150BB
:1067700030404040504068517C4F21153105410563
:10678000510571F60895019739F0880F991F880F08
:10679000991F02970197F1F70895789484B5826064
:1067A00084BD84B5816084BD85B5826085BD85B5B5
:1067B000816085BDEEE6F0E0808181608083E1E864
:1067C000F0E010828081826080838081816080839C
:1067D000E0E8F0E0808181608083E1EBF0E080819F
:1067E00084608083E0EBF0E0808181608083EAE771
:1067F000F0E08081846080838081826080838081FA
:10680000816080838081806880831092C1000895B8
:106810001F920F920FB60F9211242F933F934F9315
:106820005F936F937F938F939F93AF93BF93EF93F8
:10683000FF9380919B0690919C06892B29F0E09113
:106840009B06F0919C060995FF91EF91BF91AF9146
:106850009F918F917F916F915F914F913F912F9178
:106860000F900FBE0F901F9018951F920F920FB6AA
:106870000F9211242F933F934F935F936F937F93C6
:106880008F939F93AF93BF93EF93FF9380919D0658
:1068900090919E06892B29F0E0919D06F0919E062D
:1068A0000995FF91EF91BF91AF919F918F917F914A
:1068B0006F915F914F913F912F910F900FBE0F906D
:1068C0001F901895CF93DF93482F50E0CA018C5644
:1068D0009C4FFC01349140585C4FFA01849188230D
:1068E00069F190E0880F991FFC01EE59FC4FA591CA
:1068F000B491FC01E459FC4FC591D491662351F445
:106900002FB7F8948C91932F909589238C9388813D
:1069100089230BC0623061F42FB7F8948C91932FC8
:10692000909589238C938881832B88832FBF06C001
:106930009FB7F8948C91832B8C939FBFDF91CF915D
:106940000895482F50E0CA0188559C4FFC012491BE
:10695000CA018C569C4FFC01949140585C4FFA013F
:106960003491332309F440C0222351F1233071F0D4
:10697000243028F42130A1F0223011F514C0263043
:10698000B1F02730C1F02430D9F404C080918000E8
:106990008F7703C0809180008F7D8093800010C02E
:1069A00084B58F7702C084B58F7D84BD09C0809186
:1069B000B0008F7703C08091B0008F7D8093B000CE
:1069C000E32FF0E0EE0FFF1FE459FC4FA591B491C7
:1069D0002FB7F894662321F48C919095892302C0F7
:1069E0008C91892B8C932FBF08958093A0020895DA
:1069F000982F8E3008F09E5097708091A00282955B
:106A0000880F880F807C892B80937C0080917A008E
:106A1000806480937A0080917A0086FDFCCF20917B
:106A2000780040917900942F80E030E0282B392BBA
:106A3000C9010895CF92DF92EF92FF920F931F93B7
:106A4000CF93DF937C016B018A01C0E0D0E00FC0DF
:106A5000D6016D916D01D701ED91FC910190F0810E
:106A6000E02DC7010995C80FD91F0150104001152D
:106A7000110571F7CE01DF91CF911F910F91FF901A
:106A8000EF90DF90CF900895CF93DF930E94CD33A6
:106A90000E947129C0E0D0E00E94A32B2097E1F36F
:106AA0000E940000F9CF5058BB27AA270ED041C240
:106AB00001D230F006D220F031F49F3F11F41EF4E1
:106AC000C0C10EF4E095E7FBB6C1E92F54D280F3C4
:106AD000BA17620773078407950718F071F49EF5DB
:106AE0006CC20EF4E0950B2EBA2FA02D0B01B9014C
:106AF00090010C01CA01A0011124FF27591B99F034
:106B0000593F50F4503E68F11A16F040A22F232F3F
:106B1000342F4427585FF3CF469537952795A7958F
:106B2000F0405395C9F77EF41F16BA0B620B730B36
:106B3000840BBAF09150A1F0FF0FBB1F661F771FA7
:106B4000881FC2F70EC0BA0F621F731F841F48F45C
:106B5000879577956795B795F7959E3F08F0B3CFE2
:106B60009395880F08F09927EE0F979587950895CC
:106B7000A1D158F080E891E009F49EEFA2D128F06D
:106B800040E851E059F45EEF09C05BC116C2E92F3D
:106B9000E078F1D168F3092E052AC1F326173707EB
:106BA0004807590738F00E2E07F8E02569F0E02570
:106BB000E0640AC0EF6307F8009407FADB01B9014B
:106BC0009D01DC01CA01AD01EF934AD0B2D10AD0D8
:106BD0005F91552331F02BED3FE049E450FD49EC46
:106BE00063CF0895DF93DD27B92FBF7740E85FE3D8
:106BF0001616170648075B0710F4D92FE9D19F93A3
:106C00008F937F936F93BCD2E8E6F0E01DD191D1D2
:106C10002F913F914F915F91EED1DD2349F0905834
:106C2000A2EA2AED3FE049EC5FE3D0785D274DDF33
:106C3000DF917FC1DCD008F481E008954AD1E3956B
:106C400089C10CD076C13DD140F034D130F021F46F
:106C50005F3F19F0F0C05111B1C1F3C08CD198F36E
:106C60009923C9F35523B1F3951B550BBB27AA27CD
:106C700062177307840738F09F5F5F4F220F331F3F
:106C8000441FAA1FA9F333D00E2E3AF0E0E830D00B
:106C900091505040E695001CCAF729D0FE2F27D00E
:106CA000660F771F881FBB1F261737074807AB07DC
:106CB000B0E809F0BB0B802DBF01FF2793585F4F51
:106CC0002AF09E3F510568F0B6C078C15F3FECF3F3
:106CD000983EDCF3869577956795B795F7959F5F16
:106CE000C9F7880F911D9695879597F90895E1E06A
:106CF000660F771F881FBB1F621773078407BA07C9
:106D000020F0621B730B840BBA0BEE1F88F7E09523
:106D1000089504D06894B11151C1089534D188F018
:106D20009F5790F0B92F9927B751A0F0D1F0660F77
:106D3000771F881F991F1AF0BA95C9F712C0B13092
:106D400081F03BD1B1E0089538C1672F782F8827B3
:106D5000B85F39F0B93FCCF3869577956795B395D1
:106D6000D9F73EF490958095709561957F4F8F4F40
:106D70009F4F0895E89409C097FB3EF49095809545
:106D8000709561957F4F8F4F9F4F9923A9F0F92FF1
:106D900096E9BB279395F695879577956795B7956F
:106DA000F111F8CFFAF4BB0F11F460FF1BC06F5F55
:106DB0007F4F8F4F9F4F16C0882311F096E911C067
:106DC000772321F09EE8872F762F05C0662371F088
:106DD00096E8862F70E060E02AF09A95660F771F9C
:106DE000881FDAF7880F9695879597F90895990F78
:106DF0000008550FAA0BE0E8FEEF16161706E80785
:106E0000F907C0F012161306E407F50798F0621BA5
:106E1000730B840B950B39F40A2661F0232B242B7A
:106E2000252B21F408950A2609F4A140A6958FEF99
:106E3000811D811D089597F99F6780E870E060E0EB
:106E400008959FEF80EC0895DF93CF931F930F93E6
:106E5000FF92EF92DF927B018C01689405C0DA2EDD
:106E6000EF01C9D0FE01E894A59125913591459196
:106E70005591AEF3EF0129DEFE019701A801DA94E6
:106E800079F7DF90EF90FF900F911F91CF91DF91F5
:106E900008959F938F937F936F93FF93EF939B013D
:106EA000AC019DD0EF91FF91CFDF2F913F914F919A
:106EB0005F9195C000240A94161617061806090655
:106EC000089500240A941216130614060506089560
:106ED000B8CF59D0E8F3E894EFEFBB273FE048EC98
:106EE0005FE76B3D73078407950708F1FF279F57FE
:106EF000B25A6A4D7F40894CF04032F4BE5565422B
:106F0000704F8643FF4F0894EE1F915030F0BB0F37
:106F1000661F771F881FFF1FEBCF9EE7882332F085
:106F2000BB0F661F771F881F9A95C1F79395E09551
:106F300065C1092E0394000C11F4882352F0BB0F95
:106F400040F4BF2B11F460FF04C06F5F7F4F8F4F81
:106F50009F4F0895EF93E0FF06C0A2EA2AED3FE0BD
:106F600049EC5FEBB2DDE5DF0F90039401FC905834
:106F7000E5E9F0E08ECF57FD9058440F551F59F0CA
:106F80005F3F71F04795880F97FB991F61F09F3F16
:106F900079F087950895121613061406551FF2CF3F
:106FA0004695F1DF08C0161617061806991FF1CF8F
:106FB00086957105610508940895E894BB276627B6
:106FC0007727CB0197F9089512DF08F48FEF089522
:106FD0009B01AC0160E070E080E89FE332CE0BD013
:106FE000A8CF68DF28F06DDF18F0952309F023CFD4
:106FF00028CF1124E3CFBFDFA0F3959FD1F3950FE6
:1070000050E0551F629FF001729FBB27F00DB11D2C
:10701000639FAA27F00DB11DAA1F649F6627B00DBC
:10702000A11D661F829F2227B00DA11D621F739FA5
:10703000B00DA11D621F839FA00D611D221F749FB3
:107040003327A00D611D231F849F600D211D822FFA
:10705000762F6A2F11249F5750408AF0E1F0882341
:107060004AF0EE0FFF1FBB1F661F771F881F91504E
:107070005040A9F79E3F510570F0DDCE9FCF5F3F96
:10708000ECF3983EDCF3869577956795B795F79581
:10709000E7959F5FC1F7FE2B880F911D9695879509
:1070A00097F9089570DFE0F09E37D8F09639B8F47C
:1070B0009E3848F4672F782F8827985FF9CF8695F8
:1070C0007795679593959539D0F3B62FB1706B0F7F
:1070D000711D811D20F4879577956795939573C0F1
:1070E0008DC06CCF11F40EF4ACCE88C04CDFD0F361
:1070F0009923D9F3CEF39F57550B87FF8FD0569521
:107100009795B0E020F4660F771F881FBB1F1F9371
:107110000F9300249001A0018001F001A0E80E0F60
:107120001F1F0A1E511D601B710B8009B50B48F40F
:10713000600F711F801DB51F0E1B1F0B0A0A51091E
:1071400007C02E0F3F1F4A1F0E0F1F1F0A1E511D83
:10715000660F771F881FBB1FA695F795E795F8F672
:107160000617170708065B07211D311D411D0F91EA
:107170001F91B901842F9158880F9695879508958E
:107180009B01AC012CCFDF93D92FA3DEE695D795D9
:107190002AED3FE049E45FE3B33A620773078407EF
:1071A0009507D7952AF0A2EA49EC90688EDCC1DEFB
:1071B000E3EBF0E06EDEDD0F0BF00ADFDD0F0BF42A
:1071C0009058DF910895882371F4772321F0985027
:1071D000872B762F07C0662311F499270DC0905195
:1071E000862B70E060E02AF09A95660F771F881F63
:1071F000DAF7880F9695879597F908959F3F49F09C
:10720000915028F4869577956795B7959F5F80385C
:107210009F4F880F9695879597F908959150504004
:10722000660F771F881FD2F7089597FB092E072650
:107230000AD077FD04D049D006D000201AF470950A
:1072400061957F4F0895F6F7909581959F4F08952A
:10725000A1E21A2EAA1BBB1BFD010DC0AA1FBB1F5A
:10726000EE1FFF1FA217B307E407F50720F0A21BCC
:10727000B30BE40BF50B661F771F881F991F1A9439
:1072800069F760957095809590959B01AC01BD0163
:10729000CF01089597FB092E05260ED057FD04D087
:1072A000D7DF0AD0001C38F45095409530952195D1
:1072B0003F4F4F4F5F4F0895F6F79095809570952B
:1072C00061957F4F8F4F9F4F0895AA1BBB1B51E1C4
:1072D00007C0AA1FBB1FA617B70710F0A61BB70B46
:1072E000881F991F5A95A9F780959095BC01CD01EB
:1072F0000895EE0FFF1F0590F491E02D0994F89486
:02730000FFCFBD
:1073020025630025632563002563253269256325EE
:10731200303269006E6F2074656D7000256325310F
:107322002E356625630025632535692563002563AF
:1073320025352E32662563006D616E00737431004F
:1073420073743200737433007374340073743500D1
:107352007374360070682000636C2000767220001F
:10736200686C200061702000727462006C616E00B3
:1073720070702000706F69006163200000617420EA
:10738200002563257300256325332E3069256300AC
:107392002534692563256300256325336925630048
:1073A20025737C2563257325630020C0C0C0C0C03F
:1073B200C7C0C0C0C0C0200025342E30662563007F
:1073C200256325332E3066256300256325352E304F
:1073D2006625630025632531312E36667C256325BB
:1073E20031312E36660025632532690025332E3170
:1073F200662563007C7C766F6C74206469762072EB
:107402006174696F3A2020253569007C7C616D705A
:10741200206F66667365743A20202020202025356F
:1074220069007C7C616D702070657220766F6C746F
:107432003A202020202535690020202020202020ED
:10744200202020202000202064697361726D656411
:10745200202000206E6F2074656C20636F6D200009
:10746200206E6F206770732066697820002020628A
:10747200617474206C6F772020006C696E6B2071D0
:1074820075616C697479002573002000A306000001
:10749200E803E803E803E8039DFF0164AE472141E6
:1074A2000100000000A0051A359E04A104A404A74F
:1074B20004AF2B00070E091C1B1215383F3631246E
:1074C200232A2D70777E796C6B6265484F46415452
:1074D200535A5DE0E7EEE9FCFBF2F5D8DFD6D1C402
:1074E200C3CACD90979E998C8B8285A8AFA6A1B472
:1074F200B3BABDC7C0C9CEDBDCD5D2FFF8F1F6E323
:10750200E4EDEAB7B0B9BEABACA5A28F8881869391
:10751200949D9A2720292E3B3C35321F18111603C1
:10752200040D0A5750595E4B4C45426F68616673B1
:10753200747D7A898E878095929B9CB1B6BFB8ADD7
:10754200AAA3A4F9FEF7F0E5E2EBECC1C6CFC8DDD1
:10755200DAD3D4696E676075727B7C51565F584D81
:107562004A4344191E171005020B0C21262F283DF1
:107572003A33344E49404752555C5B7671787F6AA4
:107582006D64633E39303722252C2B0601080F1A11
:107592001D1413AEA9A0A7B2B5BCBB9691989F8A41
:1075A2008D8483DED9D0D7C2C5CCCBE6E1E8EFFA31
:1075B200FDF4F3C2C0C0C1C0C0C1C0C0C4C0C0C11C
:1075C200C0C0C1C0C0C3C0C0C1C0C0C1C0C0C5C0AE
:1075D200C0C1C0C0C1C0C000000000C52C1A3536F1
:1075E2002C662C962CB32C4C2CD42B1A2D8A2D00C5
:00000001FF
